S3150004000000000000000000000000000000000000E6
S3150007FE0080009FE580109FE580209FE5043092E4FF
S3150007FE10000053E10D00001A003092E5010053E19E
S3150007FE200A00001A68209FE5043092E4000053E1B7
S3150007FE300600001A003092E5010053E10300001A9C
S3150007FE4050209FE5003092E5013083E2003082E5DD
S3150007FE5044009FE50010A0E3001080E53CC09FE545
S3150007FE6000F08CE500F020E300F020E328009FE592
S3150007FE70001090E5011081E2001080E50000A0E384
S3150007FE800010A0E300F09CE543415254474F4C4510
S3150007FE90007E3201F87F32010C7E3201FCFF07003B
S3150007FEA0E80FFFFF00000000000000000000000050
S3150007FEB00000000000000000000000000000000035
S3150007FEC00000000000000000000000000000000025
S3150007FED00000000000000000000000000000000015
S3150007FEE00000000000000000000000000000000005
S3150007FEF000000000000000000000000000000000F5
S3150007FF0000000000000000000000000000000000E4
S3150007FF1000000000000000000000000000000000D4
S3150007FF2000000000000000000000000000000000C4
S3150007FF3000000000000000000000000000000000B4
S3150007FF4000000000000000000000000000000000A4
S3150007FF500000000000000000000000000000000094
S3150007FF600000000000000000000000000000000084
S3150007FF700000000000000000000000000000000074
S3150007FF800000000000000000000000000000000064
S3150007FF900000000000000000000000000000000054
S3150007FFA00000000000000000000000000000000044
S3150007FFB00000000000000000000000000000000034
S3150007FFC00000000000000000000000000000000024
S3150007FFD00000000000000000000000000000000014
S3150007FFE00000000000000000000000000000000004
S3150007FFF000000000000000000000000000000000F4
S3151C0000005CF09FE55CF09FE55CF09FE55CF09FE58E
S3151C0000105CF09FE500F020E358F09FE504F05EE2FB
S3151C00002000F020E304F05EE200F020E304F05EE260
S3151C00003000F020E3180050E30300001A38009FE587
S3151C000040000051E10000001A14F09FE500F05EE28A
S3151C00005000F020E304F05EE200F020E304F05EE230
S3151C00006000F020E30805001C2C00001C3400001CBA
S3151C0000705400001C5C00001C2400001C260002000E
S3151C0000800000A0E1010000FA1FB51FBD10B510BD90
S3151C000090DFF80CD0FFF7F8FF00F06AE900F017FA5A
S3151C0000A01080040003B4FFF7F1FF03BC00F016FA3E
S3151C0000B0F0402DE90040A0E10150A0E10260A0E162
S3151C0000C014709DE5090054E304F18F30200000EA0A
S3151C0000D01F0000EA060000EA080000EA0A0000EA1F
S3151C0000E00C0000EA0E0000EA100000EA120000EA0A
S3151C0000F0140000EA00F020E320129FE5170000EA36
S3151C00010000F020E318129FE5140000EA00F020E33B
S3151C00011010129FE5110000EA00F020E308129FE58B
S3151C0001200E0000EA00F020E300129FE50B0000EA37
S3151C00013000F020E3F8119FE5080000EA00F020E338
S3151C000140F0119FE5050000EA00F020E3E8119FE5A9
S3151C000150020000EA00F020E30300E0E3F080BDE8C3
S3151C00016000F020E3080091E58000C0E3080081E56B
S3151C0001700100A0E30C0081E50020A0E3010056E38A
S3151C0001800000001A402082E3000053E30000000A2E
S3151C000190012082E3000057E30400000A040057E331
S3151C0001A00500000A080057E30900001A050000EACA
S3151C0001B000F020E30C20C2E3080000EA00F020E374
S3151C0001C0042082E3050000EA00F020E3082082E315
S3151C0001D0020000EA00F020E30300E0E3DEFFFFEA92
S3151C0001E000F020E3022082E3005081E5082081E52F
S3151C0001F0080091E5800080E3080081E50000A0E38B
S3151C000200D5FFFFEA38402DE90040A0E10800A0E335
S3151C0002100030A0E30320A0E10010E0E300008DE520
S3151C0002200400A0E1A1FFFFEB3880BDE810402DE9DA
S3151C0002300020A0E10130A0E1090052E302F18F3059
S3151C000240200000EA1F0000EA060000EA080000EA97
S3151C0002500A0000EA0C0000EA0E0000EA100000EAA0
S3151C000260120000EA140000EA00F020E3AC109FE53F
S3151C000270170000EA00F020E3A4109FE5140000EA32
S3151C00028000F020E39C109FE5110000EA00F020E33B
S3151C00029094109FE50E0000EA00F020E38C109FE509
S3151C0002A00B0000EA00F020E384109FE5080000EA3A
S3151C0002B000F020E37C109FE5050000EA00F020E337
S3151C0002C074109FE5020000EA00F020E30300E0E35F
S3151C0002D01080BDE800F020E3040091E50040E0E357
S3151C0002E0000044E0000083E50000A0E3F7FFFFEAFE
S3151C0002F038402DE90040A0E10200A0E3C0FFFFEB5F
S3151C00030000F020E30D10A0E10200A0E3C6FFFFEB06
S3151C00031000009DE5040050E1F9FFFF3A3880BDE876
S3151C0003200020230320202303003023032030230333
S3151C0003300060230320602303007023032070230323
S3151C00034038402DE9AC009FE5004090E500F020E325
S3151C0003500D10A0E10100A0E3B3FFFFEB301507E38E
S3151C00036000009DE5010050E1F8FFFF3A3880BDE82A
S3151C00037084409FE584509FE5000094E5000050E30F
S3151C0003800100000A181800EB920000EB70009FE5B4
S3151C000390BC1700EB141800EB000095E5631800EB86
S3151C0003A06500A0E3751800EB682805E354109FE56B
S3151C0003B054009FE5180000EB002800E34C109FE555
S3151C0003C04C009FE5140000EB5EF07FF55EF07FF5B8
S3151C0003D06EF07FF50100A0E3C81800EB7500A0E3E2
S3151C0003E0661800EBD5FFFFEB0000A0E324109FE589
S3151C0003F0000081E5770000EBC01F240304100218DF
S3151C000400142F0118007E3201200A001C0000320144
S3151C0004100078001C007632010080320110402DE964
S3151C000420202052E20500003A1850B1E8202052E282
S3151C0004301850A0E81850B1E81850A0E8F9FFFF2A98
S3151C00044002CEB0E11850B1281850A0281800B148A7
S3151C0004501800A0481040BDE802CFB0E1043091243A
S3151C000460043080241EFF2F01822FB0E1B230D12030
S3151C0004700120D144B230C0200120C0441EFF2FE110
S3151C0004804FF0000200B5134694469646203922BF0B
S3151C000490A0E80C50A0E80C50B1F12001BFF4F7AF56
S3151C0004A0090728BFA0E80C5048BF0CC05DF804EB38
S3151C0004B0890028BF40F8042B08BF704748BF20F8A6
S3151C0004C0022B11F0804F18BF00F8012B7047044611
S3151C0004D0AFF300802046FFF7E5FD00000149182018
S3151C0004E0ABDFFEE72600020070470000101F11EE6E
S3151C0004F0011AC1E30410C1E3021BC1E34FF07FF5EF
S3151C000500101F01EE0EF0A0E1A0009FE5001090E583
S3151C000510000051E30800000A94009FE594109FE533
S3151C00052094209FE5043090E4043081E4020050E1FD
S3151C000530FBFFFFBA7CC09FE51CFF2FE17CD09FE52B
S3151C0005407C009FE50010E0E3001080E574009FE549
S3151C0005500A10A0E3081080E50C1080E50020E0E3FB
S3151C000560002080E5801081E3081080E50050E0E360
S3151C00057050609FE550709FE5048096E5088045E035
S3151C000580008087E50107A0E30518A0E30020A0E38F
S3151C000590042080E4010050E1FCFFFFBAD2F021E305
S3151C0005A028D09FE553F021E324C09FE51CFF2FE1D3
S3151C0005B0041002180076001C00FE07000078001CC0
S3151C0005C010800400140008000020230300102E01D4
S3151C0005D0108404008000001C1C009FE51C109FE575
S3151C0005E01C209FE5043090E4043081E4020050E1B5
S3151C0005F0FBFFFFBA0CC09FE51CFF2FE10076001C19
S3151C00060000FE07000078001C00FE0700B0FBF1F29C
S3151C00061002FB11011046704700000000000000009C
S3151C00062000000000000000000000000000000000A8
S3151C0006300000000000000000000000000000000098
S3151C0006400000000000000000000000000000000088
S3151C0006500000000000000000000000000000000078
S3151C000A2068640000C1000000D5030000D703000065
S3151C000A300000000000000000000000000000000094
S3151C000A40000000000000000000000000D9030000A8
S3151C000A500000000000000000DB030000EB000000AB
S3151C000A60DD030000DD030000DD030000DD030000E4
S3151C000A70DD030000DD030000DD030000DD030000D4
S3151C000A80DD030000DD030000DD030000DD030000C4
S3151C000A90DD030000DD030000DD030000DD030000B4
S3151C000AA0DD030000DD030000DD030000DD030000A4
S3151C000AB0DD030000DD030000DD030000DD03000094
S3151C000AC0DD030000DD030000DD030000DD03000084
S3151C000AD0DD030000DD030000DD030000DD03000074
S3151C000AE00348854601F00CF9004800478B0D0000B1
S3151C000AF06864000078490020486188610A69774962
S3151C000B004A61886107200861704770B5724D0026DE
S3151C000B102868401C2860000E00281AD02E606869C0
S3151C000B2006E0C1680A0E0902090A5118C160C069AB
S3151C000B300028F6D10DE0E068296888420CD8E069E7
S3151C000B40686186612269002160699047204601F030
S3151C000B50F7F86C69002CEED161480020C04670BDC8
S3151C000B605E490869C2035C4801D50122C260C2689D
S3151C000B70594889690069002A02D0411A0818704729
S3151C000B80401A704754480069704770B5FFF7E8FF74
S3151C000B90514E0546F06800281CD00023F3603269CC
S3151C000BA0B069AD1A07E0C1688A4202D8891AC160C9
S3151C000BB000E0C360C0690028F5D10BE0E068A842DC
S3151C000BC00BD82269002160699047E069B061204614
S3151C000BD001F0B6F8B469002CF0D170BD70B50646AC
S3151C000BE0FFF7BEFF3C4D04460A21286901F03AF87E
S3151C000BF0B16848432418202001F0CCF800281BD0EB
S3151C000C00B168816031690161716941617168002354
S3151C000C10C460C3614160A9680160491CA960A969D7
S3151C000C2000290CD00022CE68B4420AD2C161002A27
S3151C000C3005D0D061002070BD0020C04370BDA861E6
S3151C000C40F8E70A46C9690029EDD1D061C361F1E70D
S3151C000C5070B5064680680A2101F004F81E4D296805
S3151C000C604418202001F096F8002817D0B16881603E
S3151C000C7031690161716941617168C460416069686B
S3151C000C800160491C696069690026002909D0CA6887
S3151C000C90002394421AD2C16168611AE00020C04345
S3151C000CA070BD8661C661F7E7CA69002A08D0D36899
S3151C000CB09C4209D8C261CA699061C861816108E019
S3151C000CC0C661C861836104E00B461146CA6894423A
S3151C000CD0EAD2002070BD0000F013000000E000E026
S3151C000CE06814000008B50821002300911A46591EF5
S3151C000CF000F033F808BD00B5030001F013F8091E17
S3151C000D0006080B0D101215171E00364810E0354844
S3151C000D1020300DE034480BE03348203008E03348DF
S3151C000D2006E03248203003E0314801E030482030EC
S3151C000D304068C0430860002000BD0320C04300BDBE
S3151C000D4038B504460220FFF7CDFF69460220FFF79F
S3151C000D50D2FF0099A142F8D338BDF0B504461E4611
S3151C000D600320C043230000F0DDFF093706080B0DE6
S3151C000D701012151737001B4C10E01A4C20340DE0CE
S3151C000D80194C0BE0184C203408E0184C06E0174CA4
S3151C000D90203403E0164C01E0154C2034A568802352
S3151C000DA09D43A5600127E7600025012A00D1402547
S3151C000DB0002E00D03D43059A002A0ED0042A0FD0DF
S3151C000DC0082A09D108200543022005432160A56095
S3151C000DD0A0681843A0600020F0BD0C208543F3E7F3
S3151C000DE00420F0E7002023030030230300602303C4
S3151C000DF000702303FEE7FEE7FEE7FEE7FEE70000C2
S3151C000E00044909680160704710B52022024900F0A8
S3151C000E1053FF10BD74560000E01500008F4A131DC9
S3151C000E201060196000207047F0B58C4F0D46844643
S3151C000E308B488C498C4E3C1DFFF7F0FF002818DBB5
S3151C000E40874838600821C943864801E0761E11D0C0
S3151C000E5022688242FAD162463A6022682A60824A35
S3151C000E6003E023682B60521E04D02B688342F8D003
S3151C000E700020F0BD0846F0BD38B50D460021009196
S3151C000E800121C90601437648784C2430FFF7C6FF7A
S3151C000E90002818DBA0062918714D28352846FFF7AF
S3151C000EA0BDFF00280FDB69462846FFF7BDFF00285B
S3151C000EB009DB0098641E002802DA002CF3D103E03B
S3151C000EC0002C01D0002038BD0820C04338BDFCB51D
S3151C000ED00D460021009101910121C906014360487C
S3151C000EE0624C2430FFF79AFF002822DB5C4E610619
S3151C000EF028363046FFF792FF00281ADB371D694655
S3151C000F003046FFF791FF002813DB01A93846FFF78F
S3151C000F108BFF00280DDB0098641E400002D401984C
S3151C000F20002802DB002CEAD104E0002C02D0288029
S3151C000F300020FCBD4E4828800820C043FCBDFEB5E1
S3151C000F400C4681B2000C4B4FD21C029101909508A5
S3151C000F50454E69463846FFF7BAFF002843DB68460C
S3151C000F600188032000028143FF20013001436846AB
S3151C000F7001803846FFF780FF002834DB3D48694670
S3151C000F80401CFFF7A4FF00282DDB68460088C0071D
S3151C000F9025D0002E25D069463846FFF798FF002835
S3151C000FA021DB6846018834480140344801436846C1
S3151C000FB001803846FFF760FF002814DB2D48029994
S3151C000FC0801CFFF759FF00280DDB2A480199C01C1D
S3151C000FD0FFF752FF274E361D002804DB14E0761E51
S3151C000FE0CCD10820C043FEBD208881B23046FFF715
S3151C000FF043FF0028F7DB2068010C3046FFF73CFF57
S3151C0010000028F0DB241D6D1E002DEDD10020FEBD39
S3151C001010F0B58C4601461A48002515E04A5D030AC0
S3151C0010205A4000242346174F07E0D60702D05E001D
S3151C001030BE5B74405B1C9BB25208002AF5D10002B1
S3151C00104044406D1CA0B2ADB26545E7D3F0BD014668
S3151C001050401E80B20029FAD17047000020210118D9
S3151C0010600C1100004E3C2B1A10270000A086010014
S3151C001070ADDE000002D20000FCEFFFFF01100000F5
S3151C001080FFFF0000E0130000FFB5C00489030843FE
S3151C00109045490024454E0843716881B00860B06814
S3151C0010A0026037460C3F38680068002809D0706813
S3151C0010B00168432005F09FF8B0680168442005F0DC
S3151C0010C09AF831680120086038680068002804D046
S3151C0010D030680168492005F08EF8354D3068016886
S3151C0010E0890703D42146641CA942F8DB016809025E
S3151C0010F00BD501684E2005F07EF8306801684F203C
S3151C00110005F09DF84F2005B0F0BD39680968274EDB
S3151C001110083E00290DD00168532005F06CF8306894
S3151C0011200168542005F067F870680168552005F0C1
S3151C00113062F8AC4205D121465A2005F080F85A20A7
S3151C001140E1E770680168049801600020DBE770B570
S3151C0011500C46C504A0030543164800210543134845
S3151C0011604468256084682260C26813600368012293
S3151C0011701A600F4A006803689B0703D40B46491C78
S3151C0011809342F8DB03681B0205D501686F2005F046
S3151C00119056F86F2070BD914204D1732005F04FF8AC
S3151C0011A0732070BD002070BD0002002C28140000A6
S3151C0011B0A086010000020034F8B5FA4D0126FA4C4F
S3151C0011C076021421284600F090FD2068F7498842D3
S3151C0011D052D16168F64881424ED1A06800284BD195
S3151C0011E0E068002848D120690421F24A904204D1C3
S3151C0011F0F1486169A26906C0072188002058EF4F93
S3151C001200EF4BF04AB84210D1491C8800001968609F
S3151C001210A868401CA860C91C880027589F4204D097
S3151C0012202058904201D0B142F2DB880020589842E7
S3151C0012300DD1491C88000019E8602869401C2861EA
S3151C001240C91C88002058904201D0B142F5DB761E9D
S3151C001250B14208DC88002358934204D10019426825
S3151C001260D348824208D0002028606860E860C0200D
S3151C00127004F0E5FFC020F8BD0020F8BDF8B5CE4E41
S3151C00128008363069006884B2B0680068C7B2706AF4
S3151C0012900068C507ED0F2946DF2004F0ACFFCA48DD
S3151C0012A0CA49204088422FD105210907192040052B
S3151C0012B0C1600321090301611023C54A00210720CF
S3151C0012C0FFF745FF010004D0312004F0B8FF31219F
S3151C0012D01BE0FF23BF4A00210720FFF738FF010050
S3151C0012E004D0352004F0ABFF35210EE0C7239B004C
S3151C0012F0B94A00210B20FFF72AFF010004D03D202C
S3151C00130004F09DFF3D2100E00021002902D0E120D0
S3151C00131004F095FF3946204600F053FB010002D02D
S3151C001320E22004F08CFF002D08D1A3480078C007EA
S3151C00133004D1306A01680122114301600020F8BD06
S3151C001340F8B500209C4C0090083460690068009039
S3151C0013504007FAD5FF20053004F02FFFEF2292003C
S3151C00136060690068114600908143F9D1FF200C305A
S3151C00137004F023FF994D69462846FFF755FD0100E9
S3151C00138002D0FF24143480E000993C2421432846D3
S3151C0013900091FFF743FD010002D0FF24163474E0D0
S3151C0013A08F4E69463046FFF73FFD010002D0FF24F1
S3151C0013B019346AE08B4800990140112001433046DC
S3151C0013C00091FFF72BFD010002D0FF241C345CE0CA
S3151C0013D0854E69463046FFF727FD010002D0FF24E3
S3151C0013E0223452E000990820014330460091FFF751
S3151C0013F015FD010002D0FF24243446E01126B60157
S3151C00140069463046FFF710FD010002D0FF24273441
S3151C0014103BE00098010909010B200143304600916D
S3151C001420FFF7FCFC010002D0FF242A342DE04721E3
S3151C001430802689016120770180010091FFF7EEFC6F
S3151C001440010002D0FF2432341FE000996120B14311
S3151C001450B94380010091FFF7E1FC010002D0FF2493
S3151C001460353412E069462846FFF7DEFC010002D03F
S3151C001470FF243D3409E000992846A1430091FFF75B
S3151C001480CDFC010006D0FF243F34204604F0D7FED5
S3151C0014902046F8BD0020F8BDF8B50020009046484F
S3151C0014A001680805040F082C02D8601E044203D0EC
S3151C0014B02146FF24793438E03F4808300069002C67
S3151C0014C008D10268520C920703D002685203940F8B
S3151C0014D000E0042409060D0F032D03D9FF24294619
S3151C0014E0863422E0002D08D10168C90C890703D077
S3151C0014F00068C002850F00E00325394E6946304658
S3151C001500FFF792FC010002D0FF2490340DE00098F6
S3151C0015102101400A40022943014330460091FFF74E
S3151C0015207DFC010006D0FF249334204604F087FE80
S3151C0015302046F8BD0020F8BDF0B59C462B4B91B05B
S3151C0015401C6807466408169E179864001C600B04EA
S3151C001550BC330093AF23090C9B04C91802920325C4
S3151C001560019101223346002101E05B08491C012B35
S3151C001570FBD10E239A434907090F1143F023421E40
S3151C001580994313071B0F1C010C4307210902012257
S3151C0015908C43520214438C4351018C430C433146F9
S3151C0015A0002227E0EC7500000076000045494350F8
S3151C0015B0534752414C525443381400004C45525028
S3151C0015C054534F50444E4500F0FF000070B80000C5
S3151C0015D00001000200030002001402026808000059
S3151C0015E0DC04000000F3FFFF0418000000081118BB
S3151C0015F04908521C0129FBD10721C9038C435107F9
S3151C0016008A0B22430F2189048A439904114307221A
S3151C001610920591430122D20511430722520691439A
S3151C0016200A04FF32AB006C46BD32E250FA4A090C82
S3151C00163089186D1CAA00A1503146414360464018CA
S3151C001640401E6D1C00F00EFB0002112149042030C7
S3151C0016500843A90060506D1CA900F04860506D1C21
S3151C001660A900EF4860506D1C3420A9006050780713
S3151C001670400DA030010438020143EA4899228160DA
S3151C001680694652048918C16000214160E649086810
S3151C0016900007000FFBD111B0F0BDFEB506460020B9
S3151C0016A06946088169201C4601214002FFF7E4FBBC
S3151C0016B0010001D0DD4C71E00921DD48FFF7DCFBA0
S3151C0016C0010002D0D94C641C68E0D94801210B30BA
S3151C0016D0FFF7D2FB010002D0D44CA41C5EE0D54D12
S3151C0016E028680168012211430160992040043118C1
S3151C0016F01023082001930090CF4A23460020FFF7B1
S3151C0017001BFF010002D0C94C0E3447E0CB4C686865
S3151C00171021460268D20602D4491E0029F9DC00299A
S3151C0017200AD0C34E012128363046FFF7A5FB01001F
S3151C00173005D09924A40031E0BC4C1C342EE0BC4FCF
S3151C001740293702A93846FFF7C2FB010002D04D24F7
S3151C001750E40023E068460089000602D4641E002CBF
S3151C001760EFDC002C08D000213046FFF785FB01007A
S3151C00177006D0AE4C343411E02146AC4C31340DE06D
S3151C00178028680168490849000160A94800210B30F6
S3151C001790FFF772FB010006D0A44C4234204604F02D
S3151C0017A04EFD2046FEBD0020FEBD90B000200590DB
S3151C0017B03F20400204F09DFC04F0BDFC9B48BE305B
S3151C0017C004F0FBFC032004F0CFFCFFF7F5FC010042
S3151C0017D003D0C120800004F032FD96480838016809
S3151C0017E09248C63004F007FD04F041FD002807D0DE
S3151C0017F0FFF744FD010003D08C48CA3004F01FFDDE
S3151C0018008A48CD3004F0D9FC05A8FFF7F9FA07A8D9
S3151C001810FFF7FAFA099881B20598FFF7F9FB054616
S3151C0018200A98844CA84203D0804E2946D63692E0AC
S3151C00183004F01DFD002814D0002004F012FD7B4886
S3151C001840E63004F0BAFC04F088FCCB20800004F0DF
S3151C001850B4FCFFF775FD05000ED0744E0146EE363E
S3151C00186079E0606900684007C10FE8D01920400183
S3151C00187004F0E5FC724873E03320000104F09DFC83
S3151C00188000F060F9050003D0684E0146F23662E0AE
S3151C0018906648F43004F091FC1320A0210002FFF7E7
S3151C0018A0EBFA010002D0FF25C23512E04521C90121
S3151C0018B06448FFF7E1FA010002D0FF25C53508E0B0
S3151C0018C060480921401CFFF7D7FA010006D0FF2506
S3151C0018D0C635284604F0B3FC284601E000F0DCF8C7
S3151C0018E0050003D067260146F60034E04F48F93060
S3151C0018F004F063FC14220AA9684600F0DDF907A966
S3151C0019000EC90598FFF7C9FE050003D0474E0146D0
S3151C001910FC3620E04548FE3004F04FFC00F047F949
S3151C001920050002D00146484E15E0D120800004F087
S3151C00193044FCFFF7B1FD010005D0FF25D63528462E
S3151C00194004F07DFC02E000F0D2F80546002D0AD01A
S3151C0019503D4E2946761D304604F071FC280480193C
S3151C001960E168086006E0E16801200860D320800079
S3151C00197004F023FC04F0E5FBE0680068012801D0B4
S3151C00198004F0E5FB0025314E10E03146284600F0F8
S3151C0019907FF96D1C002911D000BF00BF00BF00BF1E
S3151C0019A000BF00BF00BF00BF00BF00BF606900686A
S3151C0019B08008C007E9D104F0DDFB46E704F0E1FB33
S3151C0019C0F4E770B5224A04461040224B224A98423C
S3151C0019D00BD17E2300215720FFF7B9FB010059D0FC
S3151C0019E04A2004F02CFC4A2070BD1C4D1C4BA842FE
S3151C0019F007D01C4DA84201D1012902D01A4DA8427C
S3151C001A0034D100215720FFF7A2FB010042D05220FF
S3151C001A1004F015FC522070BD0000181804083C0286
S3151C001A2038061818000D02180001021841020000A1
S3151C001A3001D2000040140000000004191027000009
S3151C001A4020030100B0D0000042030000A086010064
S3151C001A50F0FF000080B90000003C000280B80000C6
S3151C001A60FEFF0F0080B7000080B00000754884425E
S3151C001A7002D0401C84420DD101290BD1724A00218F
S3151C001A805720FFF764FB010004D0592004F0D7FB54
S3151C001A90592070BD002070BD70B56C4EB568746859
S3151C001AA01FE0206801280AD0002814D0B068FF2443
S3151C001AB0411B5734204604F0C2FB204670BD2089CA
S3151C001AC081B26068FFF7D8F9002808D0B068FF24F7
S3151C001AD0411B5234EEE7A1686068FFF79FF90C348E
S3151C001AE06D1E002C01D0002DDBDC002070BD70B5F6
S3151C001AF0564E3569F4681FE0206801280AD0002874
S3151C001B0014D03069FF24411BAD34204604F097FBEA
S3151C001B10204670BD208981B26068FFF7ADF90028A8
S3151C001B2008D03069FF24411BA734EEE7A168606822
S3151C001B30FFF774F90C346D1E002C01D0002DDBDC74
S3151C001B40002070BD70B5424C2068016804252943ED
S3151C001B50016000213F48FFF78FF9010001D03E4C80
S3151C001B6016E03D48401C04F028FB3A4800210B387F
S3151C001B70FFF782F9010002D0374CA41C08E069204B
S3151C001B8000214002FFF778F9010006D05324E40037
S3151C001B90204604F054FB204670BD7D20C000FFF794
S3151C001BA056FA20680168A9430160002070BD38B54B
S3151C001BB0002069460880692003214002FFF75CF972
S3151C001BC0010002D0244C1C3436E02248234919302B
S3151C001BD0FFF752F9010002D05724E4002CE01D4DFA
S3151C001BE0002124352846FFF747F9010002D01A4C7C
S3151C001BF0263421E017480B210B38FFF73DF901006D
S3151C001C0002D0154C2C3417E0154C69462846FFF7B4
S3151C001C105EF9010002D0104C34340DE06846008891
S3151C001C20002802D1641E002CEFDC002C01D0002001
S3151C001C3038BD21462D242401204604F000FB2046F5
S3151C001C4038BD000090B9000000F00002EC750000E1
S3151C001C50401400000CD20000950200000183000015
S3151C001C601027000030B50B46014600202022012417
S3151C001C7009E00D46D5409D4205D31D469540491B9E
S3151C001C802546954040191546521E002DF1DC30BDE7
S3151C001C9070B500242546002801DA0124404200299B
S3151C001CA001DA01254942FFF7DDFFAC4200D0404274
S3151C001CB0002C00D0494270BD03460B439B0703D042
S3151C001CC009E008C9121F08C0042AFAD203E00B78DF
S3151C001CD00370401C491C521EF9D27047D2B201E057
S3151C001CE00270401C491EFBD270470022F6E710B555
S3151C001CF013460A4604461946FFF7F0FF204610BD58
S3151C001D00064C0125064E05E0E36807CC2B430C3C2C
S3151C001D1098471034B442F7D3FEF7E6FEF0130000E2
S3151C001D20F013000030B47446641E2578641CAB4264
S3151C001D3000D21D46635D5B00E31830BC18470000EB
S3151C001D4010B5002823D0124B0022001F196803E08F
S3151C001D50814203D80A4649680029F9D1002A0AD0CB
S3151C001D601368841A9C4204D1006818181060104627
S3151C001D7002E0506000E01860002907D002680B1AC8
S3151C001D80934203D10B68D21802604968416010BDAA
S3151C001D906C140000F0B50B30C108C900144F0026A6
S3151C001DA0144A0FE003688B420BD38B4205D95C1A8D
S3151C001DB04318456830C3083B00E04368136002C003
S3151C001DC004E0021D10680028ECD13046002803D11F
S3151C001DD03868002801D00020F0BD064A064810606D
S3151C001DE0064A121AD208D20044C001203860D7E72E
S3151C001DF0701400006C1400006C580000686400002D
S3151C001E00211042208440088131126224C4488891E2
S3151C001E1000000000000000000000000000000000A0
S3151C001E20A0EB820000000000000000000000000083
S3151C001E30000000000000000000000000FC7F000005
S3151C001E400C00210310002103000021030C002103B8
S3151C001E5010002103140021030000000000000000F4
S3151C001E6008641018006510180410240304100218C6
S3151C001E70C01F2403142F0118302F0118382F0118E6
S3151C001E80542F0118102F011800000000000000003C
S3151C001E900000000000000000000000000000000020
S3151C001EA00000000000000000000000000000000010
S3151C001EB00000000000000000000000000000000000
S3151C001EC000000000000000000000000000000000F0
S3151C001ED000000000000000000000000000000000E0
S3151C001EE000000000000000000000000000000000D0
S3151C001EF000000000000000000000000000000000C0
S3151C001F0000000000000000000000000000000000AF
S3151C001F10000000000000000000000000000000009F
S3151C001F20000000000000000000000000000000008F
S3151C001F30000000000000000000000000000000007F
S3151C001F40000000000000000000000000000000006F
S3151C001F50000000000000000000000000000000005F
S3151C001F60000000000000000000000000000000004F
S3151C001F70000000000000000000000000000000003F
S3151C001F80000000000000000000000000000000002F
S3151C001F90000000000000000000000000000000001F
S3151C001FA0000000000000000000000000000000000F
S3151C001FB000000000000000000000000000000000FF
S3151C001FC000000000000000000000000000000000EF
S3151C001FD000000000000000000000000000000000DF
S3151C001FE000000000000000000000000000000000CF
S3151C001FF000000000000000000000000000000000BF
S3151C002000494543500B000200744000004A0700007B
S3151C002010443130325F3042000000000003112220A0
S3151C002020F00B002043020000B9390000C73900003C
S3151C002030000000000000000000000000000000007E
S3151C002040000000000000000000000000D539000060
S3151C002050000000000000000029020000E339000017
S3151C002060F1390000FF3900003D3A00003D3A0000FE
S3151C0020700D3A0000133A0000193A00001F3A0000FE
S3151C002080253A00002B3A0000313A0000373A00008E
S3151C0020903D3A00003D3A00003D3A00003D3A000042
S3151C0020A03D3A00003D3A00003D3A00003D3A000032
S3151C0020B03D3A00003D3A00003D3A00003D3A000022
S3151C0020C03D3A00003D3A00003D3A00003D3A000012
S3151C0020D03D3A00003D3A00003D3A00003D3A000002
S3151C0020E000000000000000000000000000000000CE
S3151C0020F000000000000000000000000000000000BE
S3151C00210000000000000000000000000000000000AD
S3151C002110000000000000000000000000000000009D
S3151C002120496E66360B02D10000030001042600012D
S3151C0021300001002000040020000000000005002013
S3151C002140080000008000000028040020000A00206F
S3151C00215000000000000000000000000048040020F1
S3151C002160000000000000000000000000000000004D
S3151C002170000000000000000000000000000000003D
S3151C002180010000000000000000000000000000002C
S3151C002190000000000000000000000000000000001D
S3151C0021A000F002F800F03EF80CA030C808382418DD
S3151C0021B02D18A246671EAB4654465D46AC4201D15D
S3151C0021C000F030F87E460F3E0FCCB6460126334251
S3151C0021D000D0FB1AA246AB4633431847843E000088
S3151C0021E0A43E0000103A02D378C878C1FAD8520728
S3151C0021F001D330C830C101D504680C60704700009B
S3151C0022000023002400250026103A01D378C1FBD8F0
S3151C002210520700D330C100D50B6070471FB51FBDD8
S3151C00222010B510BD03F09CFE1146FFF7F7FF00F03A
S3151C00223021F803F0B4FE03B4FFF7F2FF03BC00F071
S3151C00224017F8FEE7FEE7FEE7FEE7FEE7FEE7FEE71A
S3151C002250FEE7FEE7FEE7FEE7FEE7FEE7FEE7FEE734
S3151C002260FEE710B5FFF79CFF10BD0A4603467047F4
S3151C002270FEE77047FFF7FDFF03F040FC614E0027A9
S3151C0022803760052109077818306003F077FB03F0E7
S3151C0022900CFB03242407A08AB81EA08231685A4866
S3151C0022A008180782A08A2020C043A08231682020FB
S3151C0022B01322520289180880316853484030081886
S3151C0022C0408C524DC007C00F01D0022004E030687C
S3151C0022D04F494018808E000B287002F0C1FB03F09A
S3151C0022E03FFDA08AA7824B4A336890883546010B6E
S3151C0022F009030007000D0143907B0143424A9A18CB
S3151C0023001184464F4449396003223368520493436F
S3151C002310336000265EE038689221095CC022514376
S3151C0023204030818002F0F7FBA08A0120C043A082C6
S3151C0023302A680121344840301018018002F027FD1C
S3151C00234002F077FDA08A0720C043A08229680420DA
S3151C002350334A89188881A08A3248A08201202968BC
S3151C00236080032B4AC03A89180884A08A2E48A0826A
S3151C00237001212A6849032648803812185181A18AEE
S3151C0023802A49A18201212A68090312185181A18AAE
S3151C0023902749A18201212A68C90212185181A18AE2
S3151C0023A02449A18201212A688902101841813868B2
S3151C0023B003228030C07C520401021748081838607A
S3151C0023C08030807C296880079143400B0143761C32
S3151C0023D0F6B229600D48007886429CD303260E4C23
S3151C0023E0760400F029F838688030C07C0002001999
S3151C0023F038608030807C29688007B143400B0143DC
S3151C0024002960EEE78400002040A401008000002023
S3151C002410C0A101000004002000050020900000203F
S3151C00242040A30100FFBF0000FFDF0000FFEF00001C
S3151C002430FFF70000FFFB0000FEB5FE4D00262868D6
S3151C0024408030807C002817D10F273F0303F038FA11
S3151C002450F94C000C2168090C401AB8420CDDF748EF
S3151C002460FF218170F02141700670032003F0D2FB1E
S3151C00247020683904401820602968F14C8031887A1C
S3151C002480C87222680D2040031018808FC20A8A72F7
S3151C0024900106C90F03D18006800E01F0C5FF28680E
S3151C0024A00090407C002809D0012831D002282DD06C
S3151C0024B003282ED004282FD0052830D000980021C0
S3151C0024C0403081740098226880308446007A400629
S3151C0024D0C017DC495118898F401C4907C917491C6C
S3151C0024E0D94D084276D00022A88A8420C043A882EF
S3151C0024F0D0072168000ED54BC918001D8885002001
S3151C002500002110280ED21F231B1A0DE000F06EFBB3
S3151C002510FEBD00F0E0FBFEBD01F006FDFEBD00F0B9
S3151C002520D0FEFEBD0346103BAE8ADBB2002A07D0A6
S3151C0025301F26F643AE822768C44EBE19F38506E0F5
S3151C002540C34EAE8227681E02C04BFB189E85BD4E2D
S3151C00255000232768BF193F8CFF05FF0F01D0491CBC
S3151C002560C9B25B1CDBB20A2BF3D3002804D00529A5
S3151C0025701DD81F2802D016E0052914D9A88A002ABE
S3151C00258008D01F20C043A88223681020AF495918C1
S3151C002590C8850CE0AE48A882012023680003AB491D
S3151C0025A05918888503E0401CC0B22028A8D3521CA9
S3151C0025B0D2B2022A98D3A88A0420C043A8822268D1
S3151C0025C00020A249511888856046007A402108439C
S3151C0025D06146087221689B480818008C9D4E800431
S3151C0025E0800F02286CD00098A030007800284BD0B1
S3151C0025F0236803215803800F00908E484904964A8D
S3151C0026008B430260002723602DE0A88A0120C0436B
S3151C002610A882226800200D2149035118488403F022
S3151C00262080F98E4803F059F98249002009688031E7
S3151C002630C87702F0DBFC7F4800220068A0210A5400
S3151C0026408030C07C03220102834852040818794951
S3151C00265008608030807C216880079143400B0143D1
S3151C0026607F1CFFB221607E4800788742CDD300983C
S3151C0026707949020252186F490A60032252042168E2
S3151C0026804004914301432160216870480818C08AA0
S3151C00269001076848090F00684030C1740121817424
S3151C0026A03079002800D03CE7A88A0F20C043A882B6
S3151C0026B023680F2265484030181842843171FEBDCC
S3151C0026C0307901280BD1A88A0F20C043A882226822
S3151C0026D007215E4840301018418400203071604646
S3151C0026E0C07A544E00286046807A02D0002805D055
S3151C0026F008E0002806D002212F2001E0022130200C
S3151C00270003F016FB316808468030827A002A3CD0DA
S3151C002710012A42D00227062A52D0082ACFD1427C4F
S3151C002720530716D404231A431A404274827C403140
S3151C002730897A12015118C07F09061030090CC0B2E3
S3151C002740014301910023022200973321012003F04B
S3151C00275079FA306801468031CA7F002A56D0012A90
S3151C00276066D0032A65D0042AA9D101214030817480
S3151C002770216834480918C989C90775D02168091800
S3151C002780C9898907C90F70D01FE100224274012034
S3151C0027904031887402F097FBFEBD002640318E74D2
S3151C0027A00221312003F0C4FA02F010F902F003FDF5
S3151C0027B0A88A2C48A8822168224808184680FEBD93
S3151C0027C0427C930715D43A433A404274827C40318A
S3151C0027D0897A12015118C07F09061030090CC0B243
S3151C0027E0014301910023022200973221012003F0AC
S3151C0027F029FA30688030C07F002804D00228DED138
S3151C00280002F09AFFFEBD02F037FEFEBDAA8A022226
S3151C002810D243AA8223680D2252039B185F84AB8A7B
S3151C0028200123DB43AB8224680023A21853841DE0DA
S3151C00283027E0A5E090000020880000208C000020E6
S3151C0028408400002080A401000000003000A10100CB
S3151C002850FFE000002004002000050020A0860100E7
S3151C00286080000020FF7F00009FE0A1E00122CA77C4
S3151C002870897C4030807A090108180006000C212149
S3151C002880B1E023685A4A9B18DB89DB071ED0CF7739
S3151C002890A88A2020C043A882226820200D21490333
S3151C0028A05118088403F058F8002801D103F039F8B0
S3151C0028B03068014602468032907C4031897A00019C
S3151C0028C040180006010CD07F303049E02368484A86
S3151C0028D09A18D2899207D20F20D0012240308274D6
S3151C0028E00420C877A88A4348A882910322684048D6
S3151C0028F01018418003F030F8002801D103F011F8BC
S3151C0029003068014602468032907C4031897A00014B
S3151C00291040180006010CD07F403021E003F01CF863
S3151C002920226833495118898F8907C917491C0842DF
S3151C00293021D0316808468030C777AA8A2022D24324
S3151C002940AA82246820220D235B03E3181A84827C46
S3151C0029504031897A120151180906C07F090C503082
S3151C002960C0B20143009701910023022233210120AA
S3151C00297003F068F9FEBD3168012040318874FEBD44
S3151C002980012240308274AA8A1B4AAA822468531CDC
S3151C002990174AA21853800422CA77897C807A0901B7
S3151C0029A008180006000C64211DE0A98A124901E0E2
S3151C0029B0A98A1049A982226800211018418002F0B8
S3151C0029C0A1FF316801208031C87730680146024674
S3151C0029D08032907C4031897A000140180006D17FF4
S3151C0029E0000C7031C9B2084300970190BCE7000087
S3151C0029F080A40100FFBF0000FF7F0000002816D046
S3151C002A00012815D0002140004008491C400049B24D
S3151C002A100028FADAC00DE0221040CA17D20E52184E
S3151C002A2052095201891A1F22511A4018C0B2704706
S3151C002A30E0207047F0B503242407A18AFE49A18231
S3151C002A40002801DD012100E00021FC4A8902FC4E20
S3151C002A50891832680D277F03D219118101230021A1
S3151C002A605B02454207E0A28AF64AA2823268D21964
S3151C002A701381491C49B2002801DB024600E02A46A4
S3151C002A808A42F0DCF0BDF0B5EF4853210068012303
S3151C002A90095C0D270324EB4A5B027F032407E84DE0
S3151C002AA000290CD02621415EE84E084611300CD078
S3151C002AB00F2917D0A08AA2822868C0190381A08A70
S3151C002AC0A2822868C01903811BE03E20C043FFF781
S3151C002AD0B1FF0120FFF7AEFFA08AFF20A0820120D4
S3151C002AE080020BE03E20C043FFF7A4FF0120FFF746
S3151C002AF0A1FFA08AFF20A0820120C0022968891993
S3151C002B008884D1480068C18C491CC184F0BD30B58D
S3151C002B1003200007818ACE4B8382C94900240D6895
S3151C002B20CA4AAD182C84848A83820C685B1CA21842
S3151C002B301384828A8022D2438282096880200D22D5
S3151C002B4052038918088430BDBD480068BF49401827
S3151C002B50808E800480164042704710B503210907F9
S3151C002B608A8A8A138A82404280060D22C00D52022E
S3151C002B708318B34A1468B5482418E3828B8AB44B6D
S3151C002B808B821268591C1018C18210BDAE48006891
S3151C002B908030807A062801D00020704701207047BB
S3151C002BA070B5A94800210468227FA37D9A4201D3EF
S3151C002BB0D01A02E0BF20C01A8018C5B2E08C632868
S3151C002BC001D10121C903BF2A01D3002000E0501CFA
S3151C002BD0C0B2834202D10126B60331439A4202D1C6
S3151C002BE00122520311432943A18270BD70B5FFF720
S3151C002BF0D7FF0546FFF7CAFF002863D0924C216811
S3151C002C00087DBB285ED226228A5E632A5AD04031B2
S3151C002C10CE7C8B488D498F4B002E16D010321F2A26
S3151C002C2002681DD856182822B25E00689202401807
S3151C002C30408DC0B21043FFF7E1FE024620684421D6
S3151C002C40095A007F08181A541CE0026856183022CC
S3151C002C50B25E006892024018408E8005800D07E027
S3151C002C6056182C22B25E006892024018C08DC0B263
S3151C002C701043FFF7C3FE014620684422125A007F08
S3151C002C801018195420680577FFF75EFF1F21C842EC
S3151C002C901CDC20684422125A047F00211219995404
S3151C002CA0017FBF2901D3002100E0491C01772621A1
S3151C002CB0415E1F2907DAFFF7E6FE1F20FFF74DFFCF
S3151C002CC0FFF725FF70BD6321C18470BDFFF73CFF74
S3151C002CD0401E40B2F2E7F0B5FFF762FF0746FFF76A
S3151C002CE055FF00286FD0584E3068017DBB296AD22B
S3151C002CF02621415E632966D04030C07C504C534D22
S3151C002D00544B00280BD0103120681F2912D84119AA
S3151C002D102820085E216880024919498D11E0206827
S3151C002D2041193020085E216880024919498E89059F
S3151C002D30890D07E041192C20085E2168800249197B
S3151C002D40C98DC9B20843FFF759FE014630684422B3
S3151C002D50125A007F10181954306826210777415ED5
S3151C002D601F2902DAFFF78FFE2BE04422125A00219C
S3151C002D70D2199954017FBF2901D3002100E0491CB7
S3151C002D800177FFF7E1FE1E27FF43B84224DD3068BA
S3151C002D904030C07C002817D00420FFF74BFE0320D0
S3151C002DA00007818AFF21818201202168400249197E
S3151C002DB088843068C784FFF7C7FE401E40B2FFF701
S3151C002DC0CCFEFFF7A4FEF0BD3E20C043FFF732FE4B
S3151C002DD00120FFF72FFEECE731686320C884F0BDA5
S3151C002DE010B502F06DFD1849020C09680887CA86E1
S3151C002DF088844A8410BD10B5114A1168164BC9182F
S3151C002E00898E00244904047048081168C918C98EA3
S3151C002E10084310BD10B503200007818AFF21043129
S3151C002E208182074A00211468084BE4182184848A8D
S3151C002E3081821468E41811E0808B000001200000D8
S3151C002E4084000020FFFD00009000002040A001002F
S3151C002E50FF7F00000001002080A101006184848A9C
S3151C002E6081821468E418A184848A81821068C0183F
S3151C002E70C18410BD70B50446FFF7CCFF03210907BA
S3151C002E80888AFE488882FE4AE3061568DB0E0D26F4
S3151C002E907603AD196B858B8AFA4B8B8216680D14DB
S3151C002EA0F94BF61835848D8AFF258D820125166807
S3151C002EB0AD02F618B5848D8A0325ED438D821668FE
S3151C002EC00325F318DD848B8A88821068EF49401825
S3151C002ED0C48570BDF0B51F20FFF7CCFF032000078B
S3151C002EE0818A3021C9438182E54910230C680D2251
S3151C002EF05203A4186384838AE54B838201230C68DE
S3151C002F009B02E44D64196384838A2023DB438382FA
S3151C002F100C682023A2181384828ADF4D85825E02E8
S3151C002F200B68DA4A403A9B189E81838ADB4F87825C
S3151C002F300C687300A418A381848A85820C68A41863
S3151C002F40A684848A87820C68A2189384828A0822A3
S3151C002F50D243828209680820CB4A403289180880ED
S3151C002F60F0BDF8B5CE4F26213868415E0C124DB225
S3151C002F7029461F313F2904D21F2C02DC1F21CC42BB
S3151C002F8009DA0122E1B2D2038918818280304470A9
S3151C002F9085700120F8BDFFF7D7FD01463868B84E8D
S3151C002FA04030417632680D2149035218928AC27309
S3151C002FB032685118898A091201742846FFF7CDFD1B
S3151C002FC0FFF788FF38685321095C00290DD00321BF
S3151C002FD010230907FF22DC4209DA63004033C3844D
S3151C002FE08B8A8A82012252020AE0C4840FE00F2CCB
S3151C002FF00BDD63003C3BC3848B8A8A820122D2028E
S3151C0030003368A14959188A8401E06100C184C08CC7
S3151C00301040B2FFF70FFD6846FFF7EDFEFFF7E0FE37
S3151C003020FFF775FD386801218182803044708570F8
S3151C0030300020F8BDF0B5924D29680D267603891936
S3151C003040898A032409120818400040B2411024073B
S3151C003050A08A8C480C30A08201202A684003921951
S3151C00306010810A068A48A28AA08205D52A680020F1
S3151C00307092191081494204E001202A6880029219A3
S3151C0030801081A08A7F20C043A0822A680120921941
S3151C003090108100200122834F520206E0A38AA782D8
S3151C0030A02B689B191A81401C40B28842F6DBF0BD86
S3151C0030B0F0B5734D29680D2676038919898A032470
S3151C0030C00818400040B240102407A18A6D490C31F3
S3151C0030D0A18201212A688903921911810306002104
S3151C0030E0002B6B4AA38AA28204DA2A6892191181E0
S3151C0030F0404204E001222B6892029B191A81684AFD
S3151C003100684F12684032937B01225202002B13D067
S3151C003110A18A7F21C943A1822B6801219B19198190
S3151C003120002106E0A38AA7822B689B191A81491CD9
S3151C00313049B28142F6DBF0BDA38A5B4BA3824006F3
S3151C0031400123400EDB02C0182B689B191881A08A2C
S3151C003150A782286880190281A08A53487F30A082E2
S3151C003160286880190181F0BD0F304010704710B5DA
S3151C003170032109078A8A8A138A82C0051122C00D77
S3151C003180520283183E4A14683F482418E3828B8AED
S3151C003190424B8B821268591C1018C18210BD10B587
S3151C0031A0032109078A8A8A138A82C0050922C00D4F
S3151C0031B092028318324A146833482418E3828B8A95
S3151C0031C0364B8B821268591C1018C18210BD10B563
S3151C0031D0334C2068C27D014653074031002B14DA5C
S3151C0031E092070DD4812141560F314810FFF7D7FFA6
S3151C0031F02168822008560F304010FFF7B8FF0DE0FB
S3151C0032000F200856FFF754FF08E019200856FFF751
S3151C003210A4FC216850200856FFF70CFF2068C07DCF
S3151C00322000070CD503200007818A0821C943818227
S3151C003230134908200968144A40328918088010BDB1
S3151C00324070B5064602F03CFB154D04462868223034
S3151C00325002F0C7FD01461020C141601A30602D687E
S3151C0032602846363002F0BDFD01461020C1410F48EC
S3151C0032706A7C611A407C052A1FD019E0E0FF000019
S3151C00328084000020F38F000040A0010000A501006F
S3151C003290FFFB000080A10100FFBF0000FF7F0000B4
S3151C0032A090000020FFFD000080F7000000040020B5
S3151C0032B04004884203D2012070BDC001F9E70020FA
S3151C0032C070BDF8B5F8480068808A000418D4032637
S3151C0032D03607B08AF54FB782F54C202122680D209F
S3151C0032E04003101841846846FFF7AAFF00250128F1
S3151C0032F007D0B08AB78221680D2040030818458480
S3151C003300F8BDFFF764FFE8480121006841745321AA
S3151C003310095C00290ED081221156E64A10311F295C
S3151C00332021680AD889182823CB5E990223689A1823
S3151C003330528D09E0058345830BE08B182C21595EC1
S3151C003340236889029A18D28DD2B211430A0C0283C1
S3151C0033504183D9498182F8BDF8B5D34FD74D396819
S3151C003360D34EA0314878D64CC00707D1A88AD54879
S3151C003370A88201203268C002121910810020C87070
S3151C003380FFF7EBFB3868A03040784006400F062854
S3151C00339001D101F02BFE3168C9480818848BFFF750
S3151C0033A039FD282C43D0502C43D0782C43D0A02C4C
S3151C0033B043D0C82C43D0F02C43D00020A98A8321AB
S3151C0033C0A98232680102BB481218D184A98ABE4957
S3151C0033D0A982BE49326812181184A98AFF21A982C2
S3151C0033E001213268890212189184A98A8021C94355
S3151C0033F0A98233688022B2495B181A84AB8AD343EC
S3151C003400AB8233681818C284A88A1F20C043A882BE
S3151C00341032680C20511848853868A121095C06229F
S3151C0034200907490F511A8C4080308484F8BD01204D
S3151C003430C4E70320C2E70520C0E70720BEE7092032
S3151C003440BCE70B20BAE700B5974900230968DB43A4
S3151C0034500A46A032D0700B8402239370002240319E
S3151C003460CA75FFF77AFBFFF752FB00BD8E48002199
S3151C0034700068017781758182A121095C8030CA09A7
S3151C003480818C002A00D04900C1840020DBE700B5EE
S3151C003490854900230968DB430A46A032D0700B8499
S3151C0034A00223937000224031CA75FFF756FBFFF7C3
S3151C0034B02EFB00BD10B51446411A09D040001A1B3C
S3151C0034C0504302F0A9FC401C4010201800B210BD4D
S3151C0034D0D018C10F08184010F8E7F1B5724FA1219A
S3151C0034E038680126095C00258C4609074A0F3146B7
S3151C0034F091404CB2017F827D82B0914201D38B1ADE
S3151C00350002E0BF239B1A5B189BB28382BF2901D39F
S3151C003510002700E04F1CFFB20097BA4203D10127D7
S3151C003520BF033B438382914204D1818A0122520309
S3151C003530114381821F21029AC943614F012A23D15B
S3151C0035408030C08C00281FD16046C0091CD0604644
S3151C003550C00700D020210846FFF76CFA5748818A1D
S3151C0035605B4981825048012200689202A030417852
S3151C003570C907C91789028A184D490968C9190A81D8
S3151C00358041784906490E4170494801684C4808185B
S3151C003590808F454BC20A1868014680318A72C98CD5
S3151C0035A0002975D0062A73D1017DBB2970D24049EA
S3151C0035B00A68404951183027CF5F0246A0329178DD
S3151C0035C004290FD80323D3560620002F03DB411AE8
S3151C0035D03046884003E0411A30468840404218185D
S3151C0035E0D07043E00023DB4305290BD0002F11DDEF
S3151C0035F02021415E00291FDB032151561F2917DAA2
S3151C003600491C13E003201056002F00DB0123C018B1
S3151C003610D07028E0002F0FDA2021415E002915DC2E
S3151C003620032151561F23D94202DD491ED1701AE0CF
S3151C0036304030C6754D0116E0032151564B011A4602
S3151C00364020322025455F3946284605E003201056C2
S3151C00365042011346203B3846FFF72CFF054612480D
S3151C00366000684030C6751048006807840E4800681C
S3151C0036700146A0318A780746521C8A704037FA7D6B
S3151C003680012A06D003200856FFF767FAFFF73FFA10
S3151C003690FEBDBA88037FD3180E4AD554009A02770A
S3151C0036A0BF2A19D3002318E090000020DFFF00007A
S3151C0036B08400002040A0010001EC00000000003046
S3151C0036C000A00100FFF70000F30F00000CB0000083
S3151C0036D0FFFB000000010020531CBF882D04BF18EF
S3151C0036E0F84A2D0ED55503778030C28C521E93B2E4
S3151C0036F0C3840022CA70029DF34A012D1AD04D784C
S3151C003700ED090ED0808C83420BD103200007838ADF
S3151C0037107C23DB438382ED4804230568EC48281888
S3151C003720C38403252D07A88AEA48A882002C1DDD20
S3151C00373001201CE003230D2500201B076D03012619
S3151C003740760207E09C8A9A82E04C246864192681DA
S3151C003750401CC0B24C786407A70F0124BC408442AD
S3151C003760F0DC03200856FFF792FEFEBD0020DA4B64
S3151C00377080021843D54B1E680D277F03F61930812E
S3151C003780012200205202664208E0AB8ACE4BAB8275
S3151C003790CE4B1B68DB191A81401CC0B2002C01DB06
S3151C0037A0234600E033468342EFDC03200856FFF72E
S3151C0037B04AFEFEBDF0B5C94E00243068847584826D
S3151C0037C0FFF728FB03252D07A88A0320A882BF4FD5
S3151C0037D03868BF494018C4843068A030C47020467D
S3151C0037E0FFF7BBF9A88ABB48A88239680D2040039D
S3151C0037F009180C81A98ABA49A98239680818048152
S3151C003800F0BD00B5B54900200968A031C870FFF7A6
S3151C003810A4F900BD10B5B14C002120680177817553
S3151C00382081820221A03081704078C00701D02020FF
S3151C00383001E01F20C043FFF7FDF803200007818A23
S3151C003840A8498182206801230246A03041789B0248
S3151C003850C907C9178902C9189C4B1B680D24640328
S3151C0038601B19198141788023194341704807810F20
S3151C0038704020C8408032D0840020FFF708FE10BDCF
S3151C003880F0B5FFF761F9954F3968403148761F202E
S3151C003890FFF763F98D4C20680D256D034019828A4C
S3151C0038A0396808464030C27322685219928A12122D
S3151C0038B002741E22D243CA84C07C002847D0022030
S3151C0038C0FFF7B8F8386800260685067786751F2028
S3151C0038D0FFF7D0FA39685320425C0007002A08D04B
S3151C0038E0828AFF228282012223685202784FDB19C8
S3151C0038F09A848E82818A2021C94381822268202152
S3151C00390052191184818A784D858201272268BF034A
S3151C003910764952189781828A754E86822368721C54
S3151C0039205B189A81838A858223685B189F84838AA5
S3151C0039308682236859188A84818A0821C943818210
S3151C00394021680820624A403289180880F0BD1F2071
S3151C003950C043FFF76FF80120B2E770B50446FFF7C6
S3151C00396059FA03210907888A624B8B82574AE0065B
S3151C0039701568C00E0D267603AD196885888A5E48C3
S3151C00398088825E4D16685248361835848D8AFF2506
S3151C0039908D8201251668AD0230188584888A8B8233
S3151C0039A01068524940314018C48570BD00B5FFF7F8
S3151C0039B0CBF84A4959220968505400200877887563
S3151C0039C01C20FFF7CAFF00BD70B5FFF700FCFFF710
S3151C0039D021FA03200007818A3021C94381823B4A90
S3151C0039E0002113680D2464031B195984838A3D4BDB
S3151C0039F083821368424D5B195984384B1B68D975F1
S3151C003A0099759982838A2023DB43838213681B1949
S3151C003A101984838A344D85821468344BE418A18139
S3151C003A20848A334E86821468E418A181848A85822E
S3151C003A301468E418A184848A86821068C01881845C
S3151C003A4070BD10B5002300281CD02E4C0022A042AD
S3151C003A5000D92046521C400052B20028FADAD4176C
S3151C003A60E40EA41864096401121B1F24A21AD2B204
S3151C003A700A70082A09D2000E0006A21AD040C0B24B
S3151C003A800B7010BD0B70002010BD000ED21F0A70EB
S3151C003A9010BDF0B503242407A18A0E49A182002873
S3151C003AA001DD012100E00021174A8902074E891811
S3151C003AB032680D277F03D2191181012300215B0275
S3151C003AC045422BE000010020FFFD00008400002081
S3151C003AD040A00100808B00000170000090000020B7
S3151C003AE0FFF70000FFFB0000FFBF0000C0A40100A1
S3151C003AF0FF7F0000E0FF0000F30F00000CB0000089
S3151C003B0080A10100FFFF7F0001400000A28AFE4A3F
S3151C003B10A2823268D2191381491C49B2002801DBE2
S3151C003B20024600E02A468A42F0DCF0BDF0B50E27BC
S3151C003B300022F64DF64EFF43F64C0F23002916D0F5
S3151C003B40002809D0104609E0296889198988890640
S3151C003B508916791AC184F0BD1F461846FFF71FFB4C
S3151C003B602068C17D0909C9438907EDD1F0BD00282C
S3151C003B7001D0104601E01F461846FFF7F8FA2868E0
S3151C003B8080194088216880068016381AC884F0BDC2
S3151C003B9040000F3840B2704730B5DE4C002021681B
S3151C003BA0DA4A08851068DA4BC018808880068016A9
S3151C003BB0FFF7EEFF2168803148701068C0184088F6
S3151C003BC080068016FFF7E4FF216801220B4680332E
S3151C003BD098709A56002A01DB154600E055420028CB
S3151C003BE001DB034600E043429D4203DD0B8D0425A9
S3151C003BF02B430B85002A03DD0A8D02231A430A85F3
S3151C003C00002803DD088D012210430885CA7D900615
S3151C003C10800F13D0012820D0022821D003280CD1D4
S3151C003C20088D01218007C00FFFF780FF2068008DDB
S3151C003C30C007C00F0021FFF779FF30BD2820085EA2
S3151C003C40042801DB012100E00021042802DB800797
S3151C003C50C00FF0E7C007C00FEDE7D007C00FE9E7BC
S3151C003C60D007C00F0121E6E7F8B5FEF76DFFA94C9A
S3151C003C70A64D21680A464032507628680D235B0300
S3151C003C80C018808AD0732868C018808A0027001242
S3151C003C9010748F82C87DA24E03079F489F4AB38A21
S3151C003CA0B08203D528688018078003E02B6808209B
S3151C003CB09A181080C87D4007400F030002F07AF95D
S3151C003CC008050E1B2F43435E66451F20FEF745FF66
S3151C003CD0216850200856FFF7ADF918E01E20C04396
S3151C003CE0FEF73BFF216850200856FFF7A3F921E099
S3151C003CF02168C88429E00020FEF72FFF2068403089
S3151C003D00C07C002805D00120C043FEF793FE1F206F
S3151C003D10EEE72020FEF78EFE0020C043F5E70020CC
S3151C003D20FEF71BFF20684030C07C002805D002200F
S3151C003D30FEF780FE1E20C043DAE71F20C043FEF7B5
S3151C003D4079FE0120F4E7FFF727FF2068C07D4007B6
S3151C003D502BD4FFF7BFF820685321095C002922D019
S3151C003D60C07D81071FD56D49C207FF204039002A37
S3151C003D70B28AB08212D00120400211E02020FFF747
S3151C003D8088FE0020C043FFF784FEC0E71F20C04307
S3151C003D90FFF77FFE0120FFF77CFECBE70120C00268
S3151C003DA02A6851188884FEF7B2FEFFF719F82068B6
S3151C003DB05E30FFF720F82068877507774787878767
S3151C003DC0F8BD10B501F07CFD524909688884000CC9
S3151C003DD0488410BD7CB5064608686946C008FFF7CE
S3151C003DE030FE4C4D442229684E4C525A0B7FD21839
S3151C003DF0A054087FBF2801D3BF2000E0401C0877D1
S3151C003E0001A93068FFF71DFE694609780A01694653
S3151C003E1009790A4329680B4640339D880E7FAD19E4
S3151C003E2062550A7FBF2A01D3BF2200E0521CD2B2C0
S3151C003E300A779B889A18A054087FBF2801D3BF20F5
S3151C003E4000E0401C08777CBD70B5324A0E2314680E
S3151C003E500025E3842D4B2E4C00292BD000281868F6
S3151C003E6011D00019808880068016FFF791FE116814
S3151C003E7081268E57B0421ADA186800198088800687
S3151C003E808016401C10E00019808880068016FFF7FB
S3151C003E907FFE116881268E57B04208DD186800190E
S3151C003EA0808880068016401EFFF779F970BD106861
S3151C003EB0C58470BD0028186811D00019408880067A
S3151C003EC08016FFF765FE116882268E57B042EEDA21
S3151C003ED018680019408880068016401C10E00019DE
S3151C003EE0408880068016FFF753FE116882268E577F
S3151C003EF0B042DCDD18680019408880068016401E1A
S3151C003F00FFF735F970BD0000FFFD0000840000209E
S3151C003F1080A2010090000020F7FF000080A0010095
S3151C003F200000003000010020F0B585B00020694675
S3151C003F30FE4F08723868818A09047DD403252D0733
S3151C003F40A98A2021C943A982F94C202122680D2661
S3151C003F507603921951845321095C002911D026211C
S3151C003F60415E10311F2902D9C07D80070DD42068FF
S3151C003F70F04942182820105E226880025118498D8B
S3151C003F800CE002A8FEF737FF0AE02068E949421850
S3151C003F902C20105E226880025118C98DC9B20843B4
S3151C003FA0009001A8FFF74CF90390E04807683846D3
S3151C003FB03A3001F016FF1021C8410099401888427A
S3151C003FC001D20020C04303990090012921D0F98C0D
S3151C003FD000291ED0D849897C090181427CD227221E
S3151C003FE001991202914205D8D44A914274D9F97D9D
S3151C003FF0490671D501A96846FFF7ECFECB4A116844
S3151C004000CB7DD807CE48085E20D000281CDA401C81
S3151C0040101FE001A96846FFF7DDFE6846007A002806
S3151C00402010D0002001218003C903411803984003C6
S3151C0040300143BE48006800E002E0027F1143818212
S3151C00404005B0F0BD0120EDE7002002E00028FBDDF5
S3151C004050401EC884980740D55320475C0120B94AA6
S3151C0040604002002F01D05F0705D5A98AAA822168C4
S3151C0040708919088166E0DB07FF27002B13D026234E
S3151C004080CB5E103312D13E20C043FEF7D3FC012079
S3151C004090FEF7D0FCA88AAF82012122688902A548B6
S3151C0040A0101881844EE0C98C0F2905D0A98AAA82D2
S3151C0040B0216889190881D8E73F20FEF7BBFC002040
S3151C0040C0C043FEF7B7FCA88AAF8201202268800293
S3151C0040D098495118888435E051E0944F58072DD5DE
S3151C0040E09806800F06D0012815D0022816D0032862
S3151C0040F028D117E02820085E042801DB012100E0F6
S3151C0041000021032802DB8007C00F01E0C007C00F97
S3151C004110FFF79AFE16E0D807C00F0DE0D807C00FB0
S3151C0041200121F5E7088D01218007C00FFFF78CFEE2
S3151C0041303868008DC007C00F0021E9E7C88C40B263
S3151C004140FEF70BFDFFF73DFE784800270068478702
S3151C0041508787FEF7DCFC02A8FEF74DFE0090A88AB6
S3151C0041602020C043A8822068801947846F480068B5
S3151C004170C18C027F4906490C0A43828260E7010C06
S3151C0041807987B887FEF7C3FCA88A2020C043A8827B
S3151C0041902168002089194884E8E7F0B50320000748
S3151C0041A0818AF021C9438182614AF02114680D235A
S3151C0041B05B03E418E180818A6349818214680021CB
S3151C0041C0E4182181848AE024E44384821468E41878
S3151C0041D02184848A3224E44384821468E41861842A
S3151C0041E0848A5A4D858216680D24F3185C85838A49
S3151C0041F0574B838214684F4BE4182180848A554E92
S3151C00420086821468E4186180848A86821468E4189D
S3151C004210A180848AB41C84821668F618F180868A6A
S3151C00422084821668F6183181868A84821468E4189A
S3151C0042306181848A484C84821468E418A181848A2A
S3151C004240AC11848221261768B602FF18FE81868A65
S3151C004250832686821668F6187182868A3F4E868267
S3151C0042601668F6183183868A7F2636028682166879
S3151C004270F6187183868A848231241668A402F6187D
S3151C004280B483848AFF24043484821468E418218449
S3151C004290848A81821468E4186184848A8182146801
S3151C0042A0E418A184848A81821468E318D984838AD9
S3151C0042B00823DB43838213681E4C40341B19198068
S3151C0042C0838A274B83821368264C1B195984838A3D
S3151C0042D0214BC13B83821468234BE4186180848A7A
S3151C0042E081821468E418E185848A81821468E41842
S3151C0042F02186848A81821468E4186186848A818274
S3151C0043001468E418A186848A81821468E418E186FC
S3151C004310848A81821468E4182187848A81821468BD
S3151C004320E3185987838A0A4E20361FE09000002026
S3151C0043308400002040A0010000040020CC070000DF
S3151C00434026000000FFFD000080810000E0FF000049
S3151C004350DF3F0000FD130000C0C00000FD0F000081
S3151C004360FFFB000080A1010080A401008682146866
S3151C004370F84BE418A181848A86821468E318998410
S3151C004380838A85821068F34A40328018C185F0BD45
S3151C004390032109078A8A00228A82EF4900020968DA
S3151C0043A00D22520389188030488370470322120756
S3151C0043B0938A3F23938209070001090F08430002D1
S3151C0043C0802140300843E44909680D2252038918AC
S3151C0043D04883704710B500221146E04C07E0C3071E
S3151C0043E002D04B00E35A5A40491C89B240080028A7
S3151C0043F0F5D1104610BDF0B5D748D94D00680D2132
S3151C00440049034018868B00273C4609E0385D290A7B
S3151C0044104840FFF7DFFF29024840641C85B2A4B25E
S3151C004420B442F3D32846F0BDFEB5CB4E31680D27FA
S3151C0044307F03C919498BCB4A090A146800252246F1
S3151C00444080320192C84A0300527DD2000092224655
S3151C004450A0320292603A01F0ADFD190E1918183FF0
S3151C00446067F8FAFFF4F3F2F1F018EFEEEDECEBEA75
S3151C00447018E918E8180003200007818AC021C943DF
S3151C004480818231688020C9194883FEBD002905D068
S3151C00449001290ED0022916D0012146E2907C002863
S3151C0044A0F3D00120607401980121807C01F0DDFAB3
S3151C0044B037E20198AB4C807C012101F0D6FA2168C9
S3151C0044C0012048742DE2507A01210843507265740C
S3151C0044D001980021807CE9E7002906D001290BD030
S3151C0044E0022913D00329E3D117E003200007818A90
S3151C0044F0858201F0ECF905E003200007818A85829C
S3151C00450001F0E1F93168C91988830AE20320000722
S3151C004510818A85820198807CF4E703200007818AC2
S3151C004520858201F00DFAEDE7891E0B0001F042FDB4
S3151C0045300524314B5D050400A7E7617C02295AD28C
S3151C004540D37C012B70D8937C002B01D100299CD0E5
S3151C00455011763068C019808BE084FEF702FD0100DD
S3151C00456001D006204FE07F480521006841740321D5
S3151C00457009078A8A8D822BE1907C002802D1607CF7
S3151C004580002882D0607C107601206074FFF70EFA3A
S3151C004590C7E1507A012108435072607C714E022893
S3151C0045A00AD37248704C0560714860812081411C99
S3151C0045B0704801F012FC6575FFF706FA3068582141
S3151C0045C0095C4174ADE1607C022811D2D17C0129C1
S3151C0045D02AD8917C002901D10028ADD0624901203E
S3151C0045E04875607C1076022018E0607C022803D394
S3151C0045F000990143C9B2ABE0D17C012914D8917C46
S3151C004600002905D102E0FFF7D1FEFEBD0028FCD033
S3151C004610554901204875607C107603206074FFF7AD
S3151C0046202FF9FEF774FA7CE1B1E045E111E109E1ED
S3151C004630D0E0E9E0D4E083E037E02DE021E018E0AB
S3151C00464012E00CE008E002E0FFE7605C1FE0306867
S3151C004650C019808B605464E14348405C17E03068A5
S3151C004660C019808B404A1EE0601840780202605CCC
S3151C0046700CE03068C019808B6054000A61184870C1
S3151C0046804FE1394842185278405C1202104303210C
S3151C00469009078A8A8D8235E73068C019808B324AB1
S3151C0046A0030A5418637050543BE1607C022844D2C0
S3151C0046B000290FD0012922D00229A6D12A482B492C
S3151C0046C045750D602A4941810181491C294801F023
S3151C0046D084FB30E0002300951A4611210220019527
S3151C0046E001F0B0FA2049012048754889204A088102
S3151C0046F0904201D1002000E0401C088111E11A4AB9
S3151C0047001C4811895389405C994203D1FF21013110
S3151C004710084306E0164B994201D1002100E0491CD2
S3151C0047201181032109078A8A8D823268C1B2D21986
S3151C0047309183000A67D0012081E00021052062E7F1
S3151C004740607C8446022817D3009861460843C1B290
S3151C0047500C2058E7C0A4010084000020AE3F0000D6
S3151C004760FFFF0000900000200004002088000020AD
S3151C004770FF02000000010020480705D53368F848F1
S3151C0047801B185B8EDB0705D0D07C012809D90221BA
S3151C0047900D2038E731680818408EC107C90F08205C
S3151C0047A031E7907C002803D16046002800D12CE715
S3151C0047B0EC4B01205875607C107604206074E17502
S3151C0047C0FFF752FA03200007818A8582E6480068B3
S3151C0047D0C08C97E6507A01210843E34E5072E0E6FE
S3151C0047E09088A17D4118E148405C032109078A8A0B
S3151C0047F08D823168C9198883A07DBF2801D300200A
S3151C00480000E0401CA0758CE09188A07DD74A0B184F
S3151C004810D35CBF2801D3002000E0401CC0B2A075A9
S3151C0048200918515CBF2801D3002000E0401CA0756C
S3151C00483003200007828A85821802084362E6FFF776
S3151C004840A7FDFEBD03200007818A8582FFF7D3FDE5
S3151C00485058E60298C44E41704806400F012817D0EE
S3151C004860022803D0052835D00628EAD1607C022808
S3151C00487000D3BDE6917C002901D10028E1D0B949BD
S3151C00488001204875617C11766074FEF765FD48E071
S3151C004890607C002847D006206074FEF7E7FD40E0E8
S3151C0048A0A582FEF787FF3068014640310A7E4274B6
S3151C0048B0A03045700D7634E03068C019408B0299E3
S3151C0048C0000A4870A84E4006400F12D0012821D07D
S3151C0048D00228B6D1607C0228E2D3A548A14F056008
S3151C0048E0A44878813881411CA04801F076FA7D7570
S3151C0048F0D6E7607C0228BCD2917C002901D1002815
S3151C0049009FD0984901204875617C11766074FEF72A
S3151C00491078FF06E0607C002805D007206074FEF74F
S3151C00492079FF00208BE70098C1B201206BE630B5F9
S3151C0049308D490020096808860C464886403420723A
S3151C004940627A0B46520852006272A072E0722073A1
S3151C0049508033D873834AA073927FE2730A4660320F
S3151C0049602074D075187158710887C8862075A07573
S3151C004970107150715872E07748859071D071107221
S3151C0049808885C88550721075D07450759075507690
S3151C0049909076D0761077987518760125DD7560802F
S3151C0049A058769876D876488248738873C873087484
S3151C0049B050779077D077187010769871888618740F
S3151C0049C088828875C8750883488330BD10B5FFF783
S3151C0049D0E4FBFFF7ACFF644800688079C0070BD185
S3151C0049E003200007818A0F21C94381826249002066
S3151C0049F00968624A8918488000F0F8FA10BD70B53B
S3151C004A0000F065FF574AD188002914D0CB08C01A7C
S3151C004A100818D080107B012114280ED2584B594DF2
S3151C004A2043435B199B12D4885B1C5B109C4204DCC1
S3151C004A30D174401C0FE0C000EBE700280DD0504B92
S3151C004A40514D43435B199B12D4885B1C5B109C42E3
S3151C004A5003DBD174401E107370BD0020D07470BD72
S3151C004A6070B526213F4801F0B8F93E4C262020801F
S3151C004A704648A0800B20A07300262073E67426757A
S3151C004A80667500F024FFC000E0800025FFF7B7FF25
S3151C004A906D1CEDB2082DF9D3374A1068304B403BDC
S3151C004AA0C018C08F28210007000FE0732674012050
S3151C004AB06073A1750421E175102121766676A076B6
S3151C004AC00221E17603212177242161772021A17718
S3151C004AD00521E677C90121840B2189016184032103
S3151C004AE009078D8A0F25ED438D8212680F21D21876
S3151C004AF051841C49203108715F21C9001B4801F0F3
S3151C004B006CF91B4806601B4860812081411C1748B4
S3151C004B1001F063F970BD1448002100680A2302469F
S3151C004B20018040329371D171C172817201734173DC
S3151C004B3081730174C17341824174917401718171D5
S3151C004B40C171017241724177022242710122827047
S3151C004B50024680321172D177A0300170E7E6000060
S3151C004B6080A101000004002090000020000100200C
S3151C004B7088000020FF0200008400002080A00100A5
S3151C004B809956FCFFE6F7D3005A60DA0002D1000002
S3151C004B9070B5694D2868694E8019C18E28688019C0
S3151C004BA0008F8A044B05520F5B0FD21889065208D8
S3151C004BB0890E51188204530FC206D20E9B18840903
S3151C004BC0E40700D05B424405640FA2184009C007E5
S3151C004BD000D052429818431028688019408F8006CE
S3151C004BE0841628688019408F4005C21628688519C6
S3151C004BF03A20285EC012002900DA4942002B00DA4E
S3151C004C005B42C918002C00DA64420919002A00DA32
S3151C004C1052428918002800DA4042081880B270BD3A
S3151C004C20F0B5454D2868454A8018C18E28688018FD
S3151C004C30008F2B689B185B8F5B05DB121C0C2B688B
S3151C004C409B183A229A5E8B044E055B0F760F9B19B6
S3151C004C5089065B08890E5E188104C3065201490F3A
S3151C004C60DB0E120CC9188709FF0700D049424705FD
S3151C004C707F0FFB184009C00700D05B42C818296883
S3151C004C8043102E480818408F8006811648005D1870
S3151C004C908446401965002A4C4019246880182488CB
S3151C004CA000B2A706BF0F022F09D1640707D558000B
S3151C004CB080194118604608184019801800B2F0BDCA
S3151C004CC000B5FFF765FF81004000081880B200BDE3
S3151C004CD000B50022FDF738FF002801DA4042012208
S3151C004CE015490968154B4033C9180988C908C907ED
S3151C004CF0C90F02D04000134902E012494000403956
S3151C004D00085E002A01D0404200B200BD10B5032146
S3151C004D1009078A8A8A138A82074A80061468C30D81
S3151C004D2006482418E3828B8A074B8B821268591C0F
S3151C004D301018C18210BD00008400002040A0010094
S3151C004D4090000020FE3F0000FF7F000030B50322CC
S3151C004D501207938AFE4B93824402FE480568FE4B5B
S3151C004D60ED18EC82948A7F24640294820468E41809
S3151C004D70E182918AF949918205684C1CED18EC82F6
S3151C004D80948A918200680021C018C18230BDF0B59A
S3151C004D9003200007818AF2498182EE4901230C68AF
S3151C004DA05B03F04AA418E381838AEF4B83820123B9
S3151C004DB00C689B03A418E381838AEB4B80338382A4
S3151C004DC009230C685B02A418E382838AE74D85825B
S3151C004DD00E681424E34B4033F6183484868A858285
S3151C004DE00E68F6187484848AE14C848201260F6846
S3151C004DF07602FF183E84878A84820F68FB185E84BD
S3151C004E00838A85820D680023AD186B82858A84820D
S3151C004E100D68AD186B82858A848208688018838227
S3151C004E201124E0B20021FFF791FF641C182CF8DB5B
S3151C004E30F0BD70B503242407A08AC848A082C54DBE
S3151C004E40401C2968C74E8919C881A08A3F20C043C7
S3151C004E50A08229681420C04A8918C8811F20FFF720
S3151C004E6055FFA08A0F20C043A08229680420BA4A95
S3151C004E70403289184880A08A7F20C043A0822968B6
S3151C004E80242089190883A08ABA48A08201222B688B
S3151C004E909203B44940315B181A84A38AA0822B68FA
S3151C004EA05B185A84A28AA0822B68002259188A840D
S3151C004EB0A18AA082296889194A82A18AA0822868A7
S3151C004EC08019828270BD10B503200007818AA6490D
S3151C004ED08182A04A00231468A24964186384838AC9
S3151C004EE09E4B83821268581C5118488410BD10B5FD
S3151C004EF0032109078A8A9F4A8A8282029548036887
S3151C004F00984C1B199A828A8A9B4A8A8205230468B2
S3151C004F105B02914AA41863828B8A984B8B82072367
S3151C004F2004685B03A41863828B8A2023DB438B8271
S3151C004F3004682023A41863828B8A1023DB438B828C
S3151C004F4004681023A41863828B8A4023DB438B825C
S3151C004F5004680023A41863828C8A0C24E4438C8284
S3151C004F6000688018438210BD70B5032109078A8A20
S3151C004F70804A8A828202774803687A4C40341B191D
S3151C004F809A848A8A754B8B8205685C1C724AAD189A
S3151C004F902C838C8A8B8204680023A41863838C8AD6
S3151C004FA0774C8C820468A41823838C8A754C8C825B
S3151C004FB00468A41823838B8A0223DB438B82046830
S3151C004FC00223A41823838C8A0F24E4438C8204684E
S3151C004FD0A41863838B8AF023DB438B820068202111
S3151C004FE0801841830020FEF725F870BDF0B503201C
S3151C004FF00007818A5C498182564901230C689B0300
S3151C005000584AA2189384828A544B83820C685D1C6E
S3151C005010544AA2189584828A7F22520282820E6882
S3151C00502000244D4AB618F482868A494E86820F6839
S3151C005030AE11BF18FE82868A83820E68B618F58268
S3151C005040868A83820E68B618F482868A404E8682C9
S3151C0050500F686E11BF18FE82868A83820E68B61888
S3151C005060F582868A83820E68B618F482868A384E42
S3151C00507086820F68C614BF18FE82868A83820E68D3
S3151C005080B618F582868A83820E68B618F482868ADA
S3151C0050902F4E86820F682E11BF18FE82868A838247
S3151C0050A00E68B618F582868A83820E68B618F48254
S3151C0050B0868A274E868205260F687602BF18FE82D0
S3151C0050C0868A83820E68B618F582868A83820E6863
S3151C0050D0B618F482868A1E4E86820F688614BF18FE
S3151C0050E0FE82868A83820E68B618F582868A838239
S3151C0050F00E68B618F482868A154E868207260F68B5
S3151C0051007602BF18FE82868A83820E68B618F582DE
S3151C005110868A83820E68B618F482868A0C4E86822C
S3151C0051200F68EE10BF18FE82868A83820E68B61838
S3151C005130F582868A83820E68B618F482868A044EA5
S3151C005140868209260F687602BF18FE82868A1BE0B5
S3151C005150FFC100008400002040A00100FF7F00006A
S3151C005160FFDF0000C0A40100FFBF0000E0FF00003D
S3151C0051701FFC0000FF830000FFF00000FF0F000073
S3151C005180FF9F0000FFEF000083820E68B618F582B1
S3151C005190858A83820D68AA18D482828AFE4A8282F4
S3151C0051A00D68FE4AAA189484828A83820968FB4881
S3151C0051B008188484F0BDF8B51F20FFF7A7FD03244B
S3151C0051C02407A08A0F20C043A082F54E0720316811
S3151C0051D0F44D49194880A08A7F20C043A0823268BA
S3151C0051E02221EE48101801830020FDF723FFA08A18
S3151C0051F00820C043A08231680820491908801E2057
S3151C005200FDF7ABFC1125E8B20021FFF79FFD6D1CD5
S3151C005210172DF8DBA08AF020C043A082E048C021ED
S3151C00522000680D277F03C019C180A08ADE48A082B2
S3151C005230DB4A012113688903D84A40329B1819841A
S3151C005240A38AA082D64B1B689A185184A18AA08275
S3151C005250D34800250168D148081845822846FFF71F
S3151C00526046FED2481921006860300170A08AD04ED3
S3151C005270A682CB48711C0268CA4840381218118392
S3151C005280A18AA682C649096809184D83A18AA682E5
S3151C005290C349096809184D80A18AA682C0490968B4
S3151C0052A009188D80A18AA682BD4909680918CD8076
S3151C0052B0A18AA682BA49096809180D81A18AA68203
S3151C0052C0B7490968081845811020FFF74DFEA08ACA
S3151C0052D02020C043A082B24920200968C91908842D
S3151C0052E0A08AE81EA082AE480068C0194584A08A20
S3151C0052F0A81EA082AA4801250068C0194584AD488D
S3151C00530000F0EBFAA6480068A44940394018808F83
S3151C005310C00703D000F005FB00F0F4FAA3480022F6
S3151C00532000689F210A54A0210D549D490B689D4D70
S3151C00533080355B19DB8A1B071B0F4030C374A08AA0
S3151C005340A6820B6895481B185A84A28A924AA28286
S3151C00535001220968920308184284F8BDF0B503209F
S3151C0053600007818A924C84828D4900230D688D4AE0
S3151C005370403AAD182B83858A84820D68AD186B83E1
S3151C005380858A84820E68651CB6187580868A848216
S3151C0053900E68B618B580868A84820E68B618F580A3
S3151C0053A0868A84820E68B6183581868A84820E683F
S3151C0053B0B6187581868A84820C68A4182580848A0E
S3151C0053C0754C84826C100D68AD182C80848A7A4EBC
S3151C0053D086820D680224AD186C80858A86820D68CB
S3151C0053E0AD18AC80848A3F24E44384820C68202751
S3151C0053F0A418A781848A714C84820D683C02AD185E
S3151C005400AC81848A6E4C84820D68AD186B80858A4B
S3151C0054106C4D85820E68B6187380868A84820E68E7
S3151C005420B618B380868A85820E68B618B380868ABB
S3151C00543084820E68B618F380868A85820E68B61832
S3151C005440F380868A84820E68B6183381868A8582A2
S3151C0054500E68B6183381868A84820C68A418638108
S3151C005460848A85820C68A4186381838AFB438382A1
S3151C005470086880180780F0BDF0B503242407A08AAD
S3151C0054804B4EA682464D00202968464F403FC919FF
S3151C0054900883A08AA68229680020C9194883FFF7B9
S3151C0054A05DFFA08A4048A0820120296880033B4AF0
S3151C0054B0403289188884A08AA6822968701CC9195A
S3151C0054C04880A08A4020C043A0822A6840210D2023
S3151C0054D0400312181184A18A2021C943A1822A687B
S3151C0054E0002110180184F0BD70B503242407A18A7D
S3151C0054F02D49A1822A4D80022968284A40328918E2
S3151C0055008884A08A2A4AA2822B6800212548403812
S3151C0055101B181983A38AA2822B68521C1B185A8338
S3151C005520A28A274AA2822A6812181183A28A264AAC
S3151C005530A2822A6812181183A18A0221C943A18258
S3151C0055402A68022112181183A28A0F22D243A28230
S3151C0055502A6812185183A18AF021C943A1822A689C
S3151C005560202112185183A18A1849A1821F222B6857
S3151C00557092021B189A83A28AA18219212A6889027F
S3151C0055801018C1810020FDF755FDA08A0820C043D4
S3151C005590A082082029681BE0FFBF0000C0A40100F0
S3151C0055A08400002080A00100FF83000090000020E2
S3151C0055B0FF7F0000A0860100FDFF0000FFC0000069
S3151C0055C0FF9F0000FFF30000FFEF0000FF03000039
S3151C0055D0AB4A8918088070BDF8B5FFF779FBA94C52
S3151C0055E02168C884FFF76CFB2168A74C4884226895
S3151C0055F0A34840381018808E03258006800E02466C
S3151C005600143A00272D070C2AA04EAA8AAF822268BC
S3151C00561014D3921950861428A88AAF82206806D201
S3151C0056208019808E22689219401C908613E080197E
S3151C005630C08E22689219401CD0860CE092191086E6
S3151C005640AA8AAF8222689219D28D23689B19521C92
S3151C005650DA85602250542620085E4A8C82188C48B3
S3151C005660008C82420EDA2368854840381818808ED2
S3151C005670C00B07D10B46603318781F2802D2401C7A
S3151C005680187013E08248408C82420FDD22687C48E9
S3151C00569040381018808E800BC007C00F06D10A46F2
S3151C0056A060321078142801D9401E107060310878B9
S3151C0056B0FFF72CFBA88AAF8272482168006860300D
S3151C0056C0007889190887A88AAF8220688019408FBC
S3151C0056D021688919401C4887F8BD70B56A4D286831
S3151C0056E0674E80194088674C01072068090F603097
S3151C0056F08170FFF795FA082807DD216860318A78E2
S3151C0057000F2A02D2521C8A7009E00821C84206DA06
S3151C005710216860318878002801D0401E88700320DB
S3151C0057200007818A0F21C94381822068296860305D
S3151C00573080788919488070BDFEB5524F02263A689A
S3151C0057404032907A01280CD0002502280BD039460D
S3151C00575009688031032803D0042800D08D774D7743
S3151C0057600D779672FEBD03242407A08A494BA3829B
S3151C005770454D00202A684249403952181083A28A96
S3151C005780A3822A6851184883FFF7E8FDA08A42487D
S3151C005790A0820120296800033C4A8032891888842B
S3151C0057A0A08A4020C043A0822A6840210D204003C5
S3151C0057B0101801843868012402468030017F491C78
S3151C0057C0C9B2017700290ED0FFF706FF38680325FA
S3151C0057D002468030417F491CC9B24177022905D255
S3151C0057E040329572FEBD40329472FEBDFFF775FFC6
S3151C0057F0386802468030817F491CC9B281770229EC
S3151C00580003D2042040329072FEBD00F0A5F8002899
S3151C00581013D000F086F8214800F05FF800F072F80B
S3151C005820386801468030C477807C4031897A000113
S3151C00583040180006000CF1210BE038680146803048
S3151C005840C577807C4031897A000140180006000C1F
S3151C005850E3210843019000230222322100960120F5
S3151C00586000F0F0F903200007818A2021C9438182B8
S3151C0058700548002102680D20400310180184FEBD56
S3151C00588080A00100900000208400002080A401005C
S3151C00589000040020FF7F0000FF830000A08601009B
S3151C0058A034480079C007C00F7047324801788F22F0
S3151C0058B01140017001790178012211430170704772
S3151C0058C02C48806870472B48008980B2704703209B
S3151C0058D00007008A8005800D7047274909688031BA
S3151C0058E0897C0907090E8A002249403151188860B3
S3151C0058F008788F2210401030087008780122104357
S3151C005900087070471C4800688030807C0007000EB9
S3151C0059108100184840300818017802221143017092
S3151C0059207047154800688030807C0007000E810097
S3151C0059301048403008180178FD221140017070474C
S3151C0059400D480C49006840318030807C0007000EF1
S3151C00595080004018C06870470748064900684031F7
S3151C0059608030807C0007000E800040180079C0073C
S3151C005970C00F7047C00000309000002010B572B6F2
S3151C0059805849C869FF22120490430122920510430C
S3151C005990C86156495448486088600020544A012111
S3151C0059A0C406E40E0B46A3404409A400A4182360B5
S3151C0059B0401C40B20C28F3DB62B610BD10B50022A9
S3151C0059C01146019800F0A4F810BD10B5002211462E
S3151C0059D0019800F09DF810BD10B5002211460198E3
S3151C0059E000F096F810BD10B500221146019800F083
S3151C0059F08FF810BD10B500221146019800F088F8EA
S3151C005A0010BD10B500221146019800F081F810BD9A
S3151C005A1010B500221146019800F07AF810BD10B599
S3151C005A2000221146019800F073F810BD3148407EE3
S3151C005A30C4E73048807EC1E72E48C07EBEE72D48AD
S3151C005A40007FBBE72B48407EBFE72A48807EBCE729
S3151C005A502848C07EB9E72748007FB6E710B5002264
S3151C005A601146019800F054F810BD70B5214B024642
S3151C005A705D7E04200824954210D09D7E954202D15D
S3151C005A80052009240AE0DD7E954202D106200A245F
S3151C005A9004E01B7F934201D107200B24002905D06B
S3151C005AA000F014F8204600F011F870BD00F004F860
S3151C005AB0204600F001F870BDC206D20E01219140AD
S3151C005AC040090D4A8000801801607047C206D20E3C
S3151C005AD001219140084A40098000803280180160EB
S3151C005AE07047000004ED00E08080808000E400E048
S3151C005AF080E200E00004002000E100E010B5202157
S3151C005B003E4800F06CF920213D4800F068F910BDB4
S3151C005B1072B6BFF3408F032109078A8A00238B8242
S3151C005B20394A38491268394C1219D1863849202409
S3151C005B300A7C22430A74EFF30581304A8906890ED2
S3151C005B4014781170002C0DD191709060EFF30880C1
S3151C005B50D060EFF309801061EFF306809061EFF3DC
S3151C005B600380D0610120102906D3054610395469DB
S3151C005B708D402C43546104E0054654688D402C43EB
S3151C005B8054605370BFF3408F62B6D1780143D17015
S3151C005B90FEE7F0B5059D72B6BFF3408F1C4C40273F
S3151C005BA0267C3E432674164C26782070002E09D17E
S3151C005BB0A070A160EFF30881E160EFF30981E56154
S3151C005BC0A36121610121202806D30D462038636973
S3151C005BD085402B43636104E00B46656883401D4387
S3151C005BE0656000206070BFF3408F62B6002A03D048
S3151C005BF0E0780843E070FEE7F0BD000028040020B2
S3151C005C0048040020ADDE00008400002080A40100B2
S3151C005C1000040020F0B54C4D0A21695E00224B4E53
S3151C005C204B4B4C4F0AE0B45C5C54401E521C491E44
S3151C005C3009B2C0B2D2B2002900DA39460028F2D124
S3151C005C406981F0BDFFB581B0054604980B9E0028FE
S3151C005C5000D172B63C49487BFF2802D14B89082BE0
S3151C005C6001D3012400E00024029B5B1EFD2B52D2B3
S3151C005C70002C50D03449497D00294CD1012D02D02D
S3151C005C80002D03D004E0344800684079904242D38A
S3151C005C90FFF716FE0746010C30480068000C081A70
S3151C005CA00004000C12D02949FF228A70020A4A708D
S3151C005CB008700320FFF7AEFF2348417BFF2904D160
S3151C005CC04089082801D2002400E001242348002C26
S3151C005CD0076020D0012D24D0002D27D008240A9837
S3151C005CE0002808D01948310A06704170310C8170A1
S3151C005CF00A98FFF78FFF0A981449001D400120439C
S3151C005D00C87016480088020A8A7048700298087083
S3151C005D100420FFF77FFF0498002800D162B605B067
S3151C005D20F0BD0D4800688030847CD8E70F24D6E788
S3151C005D301CB50A46002100910B4601910146012023
S3151C005D40FFF780FF1CBD0000000400208C00002013
S3151C005D5000010020FF0200009000002088000020A7
S3151C005D6030B50E49002009780B4D4C1E11E002027D
S3151C005D70521980329074002805D0431E1375A04218
S3151C005D8003D1002302E02346F8E7431C401CD374CE
S3151C005D90C0B28842EBD330BD000500208000002035
S3151C005DA0704701E004C0091F0429FBD28B0701D5EB
S3151C005DB00280801CC90700D00270704700290BD0D6
S3151C005DC0C30702D00270401C491E022904D3830754
S3151C005DD002D50280801C891EE3E70022EEE7002222
S3151C005DE0DFE70378C2781946437812061B0219436B
S3151C005DF08378C0781B04194311430902090A00065B
S3151C005E0008437047002203098B422CD3030A8B429A
S3151C005E1011D300239C464EE003460B433CD4002280
S3151C005E2043088B4231D303098B421CD3030A8B4292
S3151C005E3001D394463FE0C3098B4201D3CB01C01A60
S3151C005E40524183098B4201D38B01C01A524143092B
S3151C005E508B4201D34B01C01A524103098B4201D319
S3151C005E600B01C01A5241C3088B4201D3CB00C01A86
S3151C005E70524183088B4201D38B00C01A52414308FE
S3151C005E808B4201D34B00C01A5241411A00D2014623
S3151C005E905241104670475DE0CA0F00D049420310BC
S3151C005EA000D34042534000229C4603098B422DD30B
S3151C005EB0030A8B4212D3FC22890112BA030A8B42B3
S3151C005EC00CD3890192118B4208D3890192118B4202
S3151C005ED004D389013AD0921100E08909C3098B4287
S3151C005EE001D3CB01C01A524183098B4201D38B01CA
S3151C005EF0C01A524143098B4201D34B01C01A52416D
S3151C005F0003098B4201D30B01C01A5241C3088B42B1
S3151C005F1001D3CB00C01A524183088B4201D38B009C
S3151C005F20C01A5241D9D243088B4201D34B00C01A26
S3151C005F305241411A00D20146634652415B1010463B
S3151C005F4001D34042002B00D54942704763465B1083
S3151C005F5000D3404201B50020C046C04602BD704772
S3151C005F60754600F023F8AE46050069465346C00840
S3151C005F70C000854618B020B5FCF777F960BC002731
S3151C005F804908B6460026C0C5C0C5C0C5C0C5C0C5E3
S3151C005F90C0C5C0C5C0C5403D49008D4670470446B6
S3151C005FA0C046C0462046FCF746F90000004870472C
S3151C005FB09400002030B47446641E2578641CAB42E1
S3151C005FC000D21D46635D5B00E31830BC18472110E8
S3151C005FD042208440088131126224C4488891000002
S3151C005FE00A0015001F00290034003E00490053001A
S3151C005FF05D00680072007C00870091009B00A60073
S3151C006000B000BA00C500CF00DA00E400EE00F900CB
S3151C00601003010D01180122012C0137014101000069
S3151C0060201100230034004600570069007A008C00DA
S3151C0060309D00AF00C000D200E300F5000601180168
S3151C00604029013B014C015D016F0180019201A301F5
S3151C006050B501C601D801E901FB010C021E020000B4
S3151C006060604000008000002014000000C4010000F5
S3151C00607074400000940000206C080000E001000041
S3151C00608000000000000000000000000000000000EE
S3151C006090000000000016000070B5784C0146503117
S3151C0060A003C4FF314531216008216160024600218D
S3151C0060B0FF32813211615161916101620168704D3B
S3151C0060C0704E083CA94208D14168B14205D1916F76
S3151C0060D0A94202D1D16FB1420AD001214902FBF774
S3151C0060E004FE206805604660FF3081308567C66700
S3151C0060F070BD62490246903205C1FF309930086076
S3151C00610010204860704710B55C48006801685C4BFD
S3151C00611099420FD141685B4A91420BD10146FF312E
S3151C00612081318C6F9C4205D1C96F914202D1C168E5
S3151C006130491CC16010BD514800680169491C0161B8
S3151C00614070474E4800684169491C416170474B487D
S3151C00615000688169491C8161704748480068FF30A6
S3151C006160813081690162704744490968FF31813178
S3151C0061700862704741480068FF308130016A8161BE
S3151C006180704710B53D48016801200831FAF7B3FD88
S3151C00619010BD70B5394D0646FF202C689D30005940
S3151C0061A00521FBF75FFD8800001946622868FF3051
S3151C0061B08130C169491CC16170BD10B52F4CA168E5
S3151C0061C00B68E2680968521E934204D9090401430C
S3151C0061D02068016210BDCA0061688850A06800680A
S3151C0061E0C00041180120091DFAF785FDA068016849
S3151C0061F0491C016010BD30B5204C22681346FF3285
S3151C00620081321569082D04D31169090401431962E9
S3151C00621030BD1269D200D218FF3201321065FF223E
S3151C006220206891321258D2001018FF300130416597
S3151C0062302068FF3081300169491C016130BD10B5F1
S3151C0062400E4C2268D369090480B21B070143980EC1
S3151C0062508018FF30013001612068C169491CC16189
S3151C00626010BD06490968FF318131486270470348F1
S3151C0062700068FF308130406A704700000C14000033
S3151C00628043415254474F4C4510402DE90040A0E174
S3151C00629088049FE5004080E5000090E5500080E200
S3151C0062A07C149FE5000081E570049FE5000090E5E5
S3151C0062B0650F80E26C149FE5000081E50800A0E3F1
S3151C0062C064149FE5000081E50000A0E34C149FE5E3
S3151C0062D0001091E5900181E540149FE5001091E5C1
S3151C0062E0940181E534149FE5001091E5980181E540
S3151C0062F028149FE5001091E5200081E51C049FE50C
S3151C006300000090E5000090E520149FE5010050E197
S3151C0063101100001A04049FE5000090E5040090E5B6
S3151C0063200C149FE5010050E10B00001AEC039FE5DD
S3151C006330000090E5F80190E5F0139FE5010050E19F
S3151C0063400500001AD4039FE5000090E5FC0190E5CA
S3151C006350DC139FE5010050E11300000A001200E364
S3151C006360B8039FE5000090E544E8FFFABC039FE5EF
S3151C006370A8139FE5001091E5000081E5B0039FE599
S3151C00638098139FE5001091E5040081E59C039FE5A9
S3151C00639088139FE5001091E5F80181E590039FE5C0
S3151C0063A078139FE5001091E5FC0181E51080BDE89E
S3151C0063B068139FE5000081E5001091E5901081E2CD
S3151C0063C05C239FE5001082E550139FE5001091E5C4
S3151C0063D0661F81E24C239FE5001082E51010A0E3A6
S3151C0063E044239FE5001082E51EFF2FE12C039FE549
S3151C0063F0000090E5000090E530139FE5010050E198
S3151C0064001800001A14039FE5000090E5040090E5AF
S3151C0064101C139FE5010050E11200001AFC029FE5C7
S3151C006420000090E5F80190E500139FE5010050E19E
S3151C0064300C00001AE4029FE5000090E5FC0190E5C3
S3151C006440EC129FE5010050E10600001ACC029FE504
S3151C006450000090E50C0090E5010080E2BC129FE56F
S3151C006460001091E50C0081E51EFF2FE1AC029FE5B3
S3151C006470000090E5100090E5010080E29C129FE56B
S3151C006480001091E5100081E51EFF2FE18C029FE5AF
S3151C006490000090E5140090E5010080E27C129FE567
S3151C0064A0001091E5140081E51EFF2FE16C029FE5AB
S3151C0064B0000090E5180090E5010080E25C129FE563
S3151C0064C0001091E5180081E51EFF2FE14C029FE5A7
S3151C0064D0000090E5980190E540129FE5001091E5BB
S3151C0064E0A00181E51EFF2FE130129FE5001091E50A
S3151C0064F0A00181E51EFF2FE120029FE5000090E52B
S3151C006500A00190E514129FE5001091E5980181E524
S3151C0065101EFF2FE110402DE900029FE5000090E5CB
S3151C006520081080E20100A0E33FE7FFEB1080BDE806
S3151C00653070402DE90040A0E1E0119FE5001091E5B7
S3151C0065409C0191E50510A0E32FE8FFFA0150A0E19C
S3151C006550C8019FE5000090E5240080E2054180E724
S3151C006560B8019FE5000090E59C0190E5010080E2E2
S3151C006570A8119FE5001091E59C0181E57080BDE89E
S3151C00658010402DE90040A0E198019FE5000090E530
S3151C006590000090E590119FE5001091E5011041E285
S3151C0065A0010050E10700009A78019FE5000090E584
S3151C0065B0000090E5000884E160119FE5001091E55C
S3151C0065C0200081E5150000EA58019FE5000090E5D2
S3151C0065D0000090E548119FE5001091E5804181E798
S3151C0065E040019FE5000090E5000090E530219FE505
S3151C0065F0002092E5800182E0041080E20100A0E305
S3151C00660009E7FFEB1C019FE5000090E5000090E503
S3151C006610010080E20C119FE5001091E5000081E568
S3151C0066201080BDE8F4209FE5002092E5902192E5BC
S3151C006630080052E30700003AE0209FE5002092E59F
S3151C006640902192E5022880E1D0309FE5003093E549
S3151C006650202083E5150000EAC0209FE5002092E576
S3151C006660902192E5B4309FE5003093E5153E83E218
S3151C006670820183E7A4209FE5002092E5902192E504
S3151C00668098309FE5003093E5153E83E2822183E036
S3151C006690041082E584209FE5002092E5902192E576
S3151C0066A0012082E274309FE5003093E5902183E55A
S3151C0066B01EFF2FE110402DE960309FE5003093E569
S3151C0066C01C3093E50F2003E20030A0E11138DFE710
S3151C0066D048409FE5004094E5114E84E2023184E770
S3151C0066E038309FE5003093E51C3093E5013083E29A
S3151C0066F028409FE5004094E51C3084E51080BDE8E9
S3151C00670018109FE5001091E5A40181E51EFF2FE1FD
S3151C00671008009FE5000090E5A40190E51EFF2FE10F
S3151C0067200000040004000400080004000C0004001F
S3151C00673043415254474F4C450000000000000000E6
S3151C0067400000000000000000000000000000000027
S3151C0067500000000000000000000000000000000017
S3151C0067600000000000000000000000000000000007
S3151C00677000000000000000000000000000000000F7
S7051C000000DE
